:020000040800F2
:1000000000000220118A00082188000823880008C7
:1000100025880008278800082988000800000000BB
:100020000000000000000000000000002B88000815
:100030002D880008000000002F8800083188000883
:10004000618A0008618A0008618A0008618A0008E4
:10005000618A0008618A0008618A0008618A0008D4
:10006000618A0008618A0008618A0008618A0008C4
:1000700035880008618A000841880008618A000804
:10008000618A0008618A0008618A0008618A0008A4
:10009000618A0008618A0008618A00084D880008AA
:1000A000618A0008618A0008618A0008618A000884
:1000B000618A0008618A0008618A0008618A000874
:1000C000618A0008618A0008618A0008618A000864
:1000D000618A000855880008618A00086188000864
:1000E00091880008618A0008618A0008618A000816
:1000F000618A0008618A0008618A0008618A000834
:10010000618A0008618A0008618A0008618A000823
:10011000618A0008618A0008B9880008618A0008BD
:10012000618A0008618A0008C5880008618A0008A1
:10013000618A0008618A0008618A0008618A0008F3
:10014000618A0008618A0008618A0008618A0008E3
:10015000618A0008618A0008D1880008618A000865
:10016000618A0008618A0008618A0008618A0008C3
:10017000618A0008618A0008618A000800000000A6
:04018000618A000888
:1001880010B5054C237833B9044B13B10448AFF3C9
:1001980000800123237010BDDC0100200000000056
:1001A80024B7000808B5034B1BB103490348AFF354
:1001B800008008BD00000000E001002024B700080E
:1001C800034613F8012B002AFBD1181A013870478F
:1001D80081F0004102E000BF83F0004330B54FEAF0
:1001E80041044FEA430594EA050F08BF90EA020F5D
:1001F8001FBF54EA000C55EA020C7FEA645C7FEAF0
:10020800655C00F0E2804FEA5454D4EB5555B8BF12
:100218006D420CDD2C4480EA020281EA030382EA83
:10022800000083EA010180EA020281EA0303362D15
:1002380088BF30BD11F0004F4FEA01314FF4801CE8
:100248004CEA113102D0404261EB410113F0004FFA
:100258004FEA03334CEA133302D0524263EB4303B1
:1002680094EA050F00F0A780A4F10104D5F1200E4F
:100278000DDB02FA0EFC22FA05F2801841F10001AA
:1002880003FA0EF2801843FA05F359410EE0A5F17E
:1002980020050EF1200E012A03FA0EFC28BF4CF0AF
:1002A800020C43FA05F3C01851EBE37101F0004565
:1002B80007D54FF0000EDCF1000C7EEB00006EEB72
:1002C8000101B1F5801F1BD3B1F5001F0CD34908FC
:1002D8005FEA30004FEA3C0C04F101044FEA445253
:1002E80012F5800F80F09A80BCF1004F08BF5FEADA
:1002F800500C50F1000041EB045141EA050130BDBA
:100308005FEA4C0C404141EB010111F4801FA4F15C
:100318000104E9D191F0000F04BF01460020B1FAB1
:1003280081F308BF2033A3F10B03B3F120020CDAE9
:100338000C3208DD02F1140CC2F10C0201FA0CF0C7
:1003480021FA02F10CE002F11402D8BFC2F1200C2C
:1003580001FA02F120FA0CFCDCBF41EA0C019040E2
:10036800E41AA2BF01EB0451294330BD6FEA04042B
:100378001F3C1CDA0C340EDC04F11404C4F1200216
:1003880020FA04F001FA02F340EA030021FA04F328
:1003980045EA030130BDC4F10C04C4F1200220FA7F
:1003A80002F001FA04F340EA0300294630BD21FABD
:1003B80004F0294630BD94F0000F83F4801306BF83
:1003C80081F480110134013D4EE77FEA645C18BF77
:1003D8007FEA655C29D094EA050F08BF90EA020F0E
:1003E80005D054EA000C04BF1946104630BD91EA06
:1003F800030F1EBF0021002030BD5FEA545C05D109
:100408004000494128BF41F0004130BD14F5800447
:100418003CBF01F5801130BD01F0004545F0FE41BB
:1004280041F470014FF0000030BD7FEA645C1ABFF0
:10043800194610467FEA655C1CBF0B46024650EA27
:10044800013406BF52EA033591EA030F41F4002153
:1004580030BD00BF90F0000F04BF0021704730B5D9
:100468004FF4806404F132044FF000054FF00001AE
:1004780050E700BF90F0000F04BF0021704730B56F
:100488004FF4806404F1320410F0004548BF404244
:100498004FF000013EE700BF42004FEAE2014FEA99
:1004A80031014FEA02701FBF12F07F4393F07F4F74
:1004B80081F06051704792F0000F14BF93F07F4FA6
:1004C800704730B54FF4607401F0004521F00041E9
:1004D80020E700BF50EA010208BF704730B54FF06F
:1004E80000050AE050EA010208BF704730B511F074
:1004F800004502D5404261EB41014FF4806404F1AC
:1005080032045FEA915C3FF4DCAE4FF003025FEA2D
:10051800DC0C18BF03325FEADC0C18BF033202EBB5
:10052800DC02C2F1200300FA03FC20FA02F001FA0F
:1005380003FE40EA0E0021FA02F11444C1E600BFAE
:1005480070B54FF0FF0C4CF4E06C1CEA11541DBF61
:100558001CEA135594EA0C0F95EA0C0F00F0DEF82C
:100568002C4481EA030621EA4C5123EA4C5350EA11
:10057800013518BF52EA033541F4801143F4801362
:1005880038D0A0FB02CE4FF00005E1FB02E506F0F3
:100598000042E0FB03E54FF00006E1FB03569CF048
:1005A800000F18BF4EF0010EA4F1FF04B6F5007F4E
:1005B80064F5407404D25FEA4E0E6D4146EB0606C0
:1005C80042EAC62141EA55514FEAC52040EA5E5049
:1005D8004FEACE2EB4F1FD0C88BFBCF5E06F1ED8F3
:1005E800BEF1004F08BF5FEA500E50F1000041EB2A
:1005F800045170BD06F0004646EA010140EA0200D7
:1006080081EA0301B4EB5C04C2BFD4EB0C0541EAF8
:10061800045170BD41F480114FF0000E013C00F30D
:10062800AB8014F1360FDEBF002001F0004170BD31
:10063800C4F10004203C35DA0C341BDC04F114044A
:10064800C4F1200500FA05F320FA04F001FA05F2D6
:1006580040EA020001F0004221F0004110EBD370A3
:1006680021FA04F642EB06015EEA430E08BF20EACF
:10067800D37070BDC4F10C04C4F1200500FA04F372
:1006880020FA05F001FA04F240EA020001F0004104
:1006980010EBD37041F100015EEA430E08BF20EA77
:1006A800D37070BDC4F1200500FA05F24EEA020EBF
:1006B80020FA04F301FA05F243EA020321FA04F0EE
:1006C80001F0004121FA04F220EA020000EBD370A5
:1006D8005EEA430E08BF20EAD37070BD94F0000FA5
:1006E8000FD101F00046400041EB010111F4801FD9
:1006F80008BF013CF7D041EA060195F0000F18BF8A
:10070800704703F00046520043EB030313F4801FC5
:1007180008BF013DF7D043EA0603704794EA0C0F7F
:100728000CEA135518BF95EA0C0F0CD050EA410695
:1007380018BF52EA4306D1D181EA030101F0004112
:100748004FF0000070BD50EA410606BF104619463A
:1007580052EA430619D094EA0C0F02D150EA013646
:1007680013D195EA0C0F05D152EA03361CBF104687
:1007780019460AD181EA030101F0004141F0FE4126
:1007880041F470014FF0000070BD41F0FE4141F4AA
:10079800780170BD70B54FF0FF0C4CF4E06C1CEAAA
:1007A80011541DBF1CEA135594EA0C0F95EA0C0F5F
:1007B80000F0A7F8A4EB050481EA030E52EA03351A
:1007C8004FEA013100F088804FEA03334FF080553B
:1007D80045EA131343EA12634FEA022245EA111568
:1007E80045EA10654FEA00260EF000419D4208BF19
:1007F800964244F1FD0404F5407402D25B084FEAC6
:100808003202B61A65EB03055B084FEA32024FF471
:1008180080104FF4002CB6EB020E75EB030E22BFCE
:10082800B61A754640EA0C005B084FEA3202B6EB8E
:10083800020E75EB030E22BFB61A754640EA5C003D
:100848005B084FEA3202B6EB020E75EB030E22BFCD
:10085800B61A754640EA9C005B084FEA3202B6EBCE
:10086800020E75EB030E22BFB61A754640EADC008D
:1008780055EA060E18D04FEA051545EA16754FEAEF
:1008880006164FEAC30343EA52734FEAC2025FEA0D
:100898001C1CC0D111F4801F0BD141EA00014FF09C
:1008A80000004FF0004CB6E711F4801F04BF01436D
:1008B8000020B4F1FD0C88BFBCF5E06F3FF6AFAE89
:1008C800B5EB030C04BFB6EB020C5FEA500C50F119
:1008D800000041EB045170BD0EF0004E4EEA11319C
:1008E80014EB5C04C2BFD4EB0C0541EA045170BDA3
:1008F80041F480114FF0000E013C90E645EA060EE7
:100908008DE60CEA135594EA0C0F08BF95EA0C0F14
:100918003FF43BAF94EA0C0F0AD150EA01347FF45C
:1009280034AF95EA0C0F7FF425AF104619462CE733
:1009380095EA0C0F06D152EA03353FF4FDAE104696
:10094800194622E750EA410618BF52EA43067FF4E7
:10095800C5AE50EA41047FF40DAF52EA43057FF477
:10096800EBAE12E74FF0FF3C06E000BF4FF0010C82
:1009780002E000BF4FF0010C4DF804CD4FEA410CE6
:100988007FEA6C5C4FEA430C18BF7FEA6C5C1BD0B3
:1009980001B050EA410C0CBF52EA430C91EA030F34
:1009A80002BF90EA020F0020704710F1000F91EA91
:1009B800030F58BF994208BF90422CBFD8176FEA5F
:1009C800E37040F0010070474FEA410C7FEA6C5C2D
:1009D80002D150EA013C07D14FEA430C7FEA6C5C34
:1009E800D6D152EA033CD3D05DF8040B704700BF60
:1009F8008446104662468C461946634600E000BFAE
:100A080001B5FFF7B7FF002848BF10F1000F01BD7F
:100A18004DF808EDFFF7F4FF0CBF012000205DF84A
:100A280008FB00BF4DF808EDFFF7EAFF34BF0120CF
:100A380000205DF808FB00BF4DF808EDFFF7E0FF68
:100A480094BF012000205DF808FB00BF4DF808EDB9
:100A5800FFF7CEFF94BF012000205DF808FB00BF20
:100A68004DF808EDFFF7C4FF34BF012000205DF802
:100A780008FB00BF4FEA410C7FEA6C5C02D150EAE8
:100A8800013C0AD14FEA430C7FEA6C5C02D152EA7E
:100A9800033C02D14FF0000070474FF0010070474F
:100AA8004FEA410212F5001215D211D56FF478738E
:100AB800B3EB625212D94FEAC12343F0004343EA31
:100AC800505311F0004F23FA02F018BF404270470C
:100AD8004FF00000704750EA013005D111F0004096
:100AE80008BF6FF0004070474FF00000704700BF2C
:100AF80080F0004002E000BF81F0004142001FBFCB
:100B08005FEA410392EA030F7FEA226C7FEA236CD3
:100B18006AD04FEA1262D2EB1363C1BFD2184140C8
:100B280048404140B8BF5B42192B88BF704710F05E
:100B3800004F40F4000020F07F4018BF404211F001
:100B4800004F41F4000121F07F4118BF494292EA69
:100B5800030F3FD0A2F1010241FA03FC10EB0C0095
:100B6800C3F1200301FA03F100F0004302D5494222
:100B780060EB4000B0F5000F13D3B0F1807F06D3CF
:100B880040084FEA310102F10102FE2A51D2B1F1C7
:100B9800004F40EBC25008BF20F0010040EA0300BC
:100BA8007047490040EB000010F4000FA2F1010269
:100BB800EDD1B0FA80FCACF1080CB2EB0C0200FAF3
:100BC8000CF0AABF00EBC25052421843BCBFD04041
:100BD8001843704792F0000F81F4000106BF80F4BB
:100BE80000000132013BB5E74FEA41037FEA226C7E
:100BF80018BF7FEA236C21D092EA030F04D092F049
:100C0800000F08BF0846704790EA010F1CBF00207C
:100C1800704712F07F4F04D1400028BF40F00040D9
:100C2800704712F100723CBF00F50000704700F0F9
:100C3800004343F0FE4040F4000070477FEA226220
:100C480016BF08467FEA23630146420206BF5FEAF1
:100C5800412390EA010F40F4800070474FF00003F1
:100C680004E000BF10F0004348BF40425FEA000CB8
:100C780008BF704743F0964301464FF000001CE060
:100C880050EA010208BF70474FF000030AE000BFB6
:100C980050EA010208BF704711F0004302D54042F4
:100CA80061EB41015FEA010C02BF84460146002066
:100CB80043F0B64308BFA3F18053A3F50003BCFA81
:100CC8008CF2083AA3EBC25310DB01FA02FC63442E
:100CD80000FA02FCC2F12002BCF1004F20FA02F235
:100CE80043EB020008BF20F00100704702F1200228
:100CF80001FA02FCC2F1200250EA4C0021FA02F289
:100D080043EB020008BF20EADC7070474FF0FF3C5D
:100D180006E000BF4FF0010C02E000BF4FF0010CED
:100D28004DF804CD4FEA40024FEA41037FEA226CB6
:100D380018BF7FEA236C11D001B052EA530C18BFD8
:100D480090EA010F58BFB2EB030088BFC81738BF3D
:100D58006FEAE17018BF40F0010070477FEA226C2B
:100D680002D15FEA402C05D17FEA236CE4D15FEA27
:100D7800412CE1D05DF8040B704700BF844608465B
:100D88006146FFE70FB5FFF7C9FF002848BF10F11C
:100D9800000F0FBD4DF808EDFFF7F4FF0CBF012061
:100DA80000205DF808FB00BF4DF808EDFFF7EAFFEB
:100DB80034BF012000205DF808FB00BF4DF808EDA6
:100DC800FFF7E0FF94BF012000205DF808FB00BF9B
:100DD8004DF808EDFFF7D2FF94BF012000205DF821
:100DE80008FB00BF4DF808EDFFF7C8FF34BF01202E
:100DF80000205DF808FB00BF42000ED2B2F1FE4FA2
:100E08000BD34FF09E03B3EB126209D44FEA0023D1
:100E180043F0004323FA02F070474FF00000704798
:100E280012F1610F01D1420202D14FF0FF30704739
:100E38004FF00000704700BF53B94AB9002908BFF6
:100E480000281CBF4FF0FF314FF0FF3000F07AB997
:100E5800ADF1080C6DE904CE00F006F8DDF804E009
:100E6800DDE9022304B070472DE9F0478C460E46B1
:100E78000446089D002B50D18A4217466CD9B2FA15
:100E880082FEBEF1000F0BD0CEF1200C01FA0EF657
:100E980020FA0CFC02FA0EF74CEA060C00FA0EF4E3
:100EA8003A0CBCFBF2F9BBB202FB19CC09FB03FA02
:100EB8004FEA144848EA0C46B2450AD9F61909F12E
:100EC800FF3180F02581B24540F22281A9F1020963
:100ED8003E44A6EB0A06B6FBF2F002FB106600FBE6
:100EE80003F3A4B244EA0644A34209D9E41900F181
:100EF800FF3280F00B81A34240F2088102383C4463
:100F08000021E41A40EA0940002D62D0002324FAA7
:100F18000EF42C606B60BDE8F0878B4207D9002D7A
:100F280055D0002185E841000846BDE8F087B3FAAE
:100F380083F1002940F08F80B34202D3824200F24D
:100F4800FC80841A66EB03060120B446002D40D0CD
:100F580085E81010BDE8F08712B90127B7FBF2F752
:100F6800B7FA87FEBEF1000F35D10121F61B4FEA13
:100F7800174C1FFA87F8B6FBFCF20CFB126608FB4D
:100F880002F0230C43EA0646B04207D9F61902F1EB
:100F9800FF3302D2B04200F2D2801A46361AB6FBAC
:100FA800FCF00CFB106608FB00F8A3B243EA064409
:100FB800A04507D9E41900F1FF3302D2A04500F299
:100FC800B9801846A4EB080440EA02409CE7294689
:100FD8002846BDE8F08707FA0EF7CEF1200326FA77
:100FE80003F24FEA174CB2FBFCF11FFA87F80CFB2F
:100FF800112206FA0EF620FA03F301FB08F933432F
:101008001E0C46EA0246B14500FA0EF409D9F61953
:1010180001F1FF3280F08C80B14540F289800239BD
:101028003E44A6EB0906B6FBFCF00CFB106200FB85
:1010380008F99EB246EA0246B14507D9F61900F109
:10104800FF3371D2B1456FD902383E44A6EB090689
:1010580040EA01418FE7C1F1200722FA07F88B40E7
:1010680048EA030326FA07F44FEA134EB4FBFEF9E5
:101078001FFA83FC0EFB19448E4020FA07F809FB7F
:101088000CFA48EA06084FEA184646EA0444A2451C
:1010980002FA01F200FA01F608D9E41809F1FF3062
:1010A80044D2A24542D9A9F102091C44A4EB0A047E
:1010B800B4FBFEF00EFB104400FB0CFC1FFA88F892
:1010C80048EA0444A44507D9E41800F1FF3E29D2B0
:1010D800A44527D902381C4440EA0940A0FB0289EC
:1010E800A4EB0C0CCC45C246CE4615D312D055B154
:1010F800B6EB0A036CEB0E0606FA07F7CB401F4364
:10110800CE402F606E600021BDE8F0871046F7E6FC
:101118008946DEE64645EAD2B8EB020A69EB030ED9
:101128000138E4E77046D7E718468FE78146BDE700
:10113800114676E702383C4444E7084606E7023A97
:101148003E442BE7704700BF38B50E4B054618786C
:101158004FF47A73B3FBF0F30B4A1068B0FBF3F06B
:1011680000F0AAF8044658B90F2D09D802462946B6
:101178004FF0FF3000F05EF8044B20461D6038BD8C
:10118800012038BD000000200800002004000020D5
:1011980008B50B4B03201A6842F400721A601A68EB
:1011A80042F480621A601A6842F480721A6000F091
:1011B8002FF80020FFF7C8FF07F0DEF9002008BD70
:1011C800003C0240034A044B11681B780B4413602F
:1011D800704700BF9002002000000020014B1868F3
:1011E800704700BF9002002037B50190FFF7F6FF67
:1011F8000546019C631C1EBF044B1B78E418FFF7CF
:10120800EDFF401BA042FAD303B030BD0000002020
:10121800074A0002D36800F4E06023F4E0631B048B
:101228001B0C43F0BF6343F400330343D3607047A0
:1012380000ED00E0174B30B5DC68C4F30224C4F1BC
:101248000703251D042B28BF0423062D4FF0010595
:1012580098BF002405FA03F303F1FF3388BF033C6A
:101268001940A14005FA04F4013C2240002842EA52
:1012780001024FEA0212A9BF00F16040064BD2B248
:1012880000F56140BBBF00F00F00D2B280F8002328
:101298001A5430BD00ED00E014ED00E0002808DB32
:1012A8000123420900F01F0003FA00F0014B43F844
:1012B8002200704700E100E00138B0F1807F0AD2D7
:1012C800F021064B064A586082F8231000200722B6
:1012D80098601A6070470120704700BF10E000E076
:1012E80000ED00E018210368DAB2103AB2FBF1F21F
:1012F80023F47F73054923F00303032A895C88BF1D
:1013080004338365C165806D704700BF40B700082E
:1013180070B50446FFF762FF0546002C71D0002324
:1013280084F834300223226884F83530136823F0B7
:101338000103136021680B68D8073BD40B68324D52
:1013480062681D40A368A0691343E26813432269D9
:10135800134362691343E26903431343226A134345
:10136800626A2B43042A01BFE56A266B35432B4387
:101378000B604B69042A23F0070343EA02030BD1ED
:10138800A26AE56A13433DB1F8B9012A2ED001D308
:10139800022A01D1EA012CD44B612046FFF7A2FFB3
:1013A8003F23E26D9340836000200123606584F849
:1013B800353070BDFFF712FF401B0528BAD920232E
:1013C8000320636584F8350070BDB0F5005F14D163
:1013D800032AE1D801A050F822F000BFFB1300084F
:1013E8009D130008FB130008F5130008B5F1C07F32
:1013F800D2D1402301206365E4E7022AF9D9032A00
:10140800C7E7012070BD00BF3F8010F070B590F8AD
:101418003440012C33D0012480F8344090F8354012
:10142800866D012C4FF000054FF0020425D180F89D
:10143800354004684565256825F480252560636086
:101448008368402B4FF03F030EBFA260A160E260AB
:10145800C26D08BFE1609340B360236843F0160390
:101468002360036C1BB1236843F0080323602368DF
:10147800002043F00103236070BD80F8345002203F
:1014880070BD90F83530022B03D0802343650120CE
:1014980070470523026880F835301368002023F070
:1014A80001031360704700000023F7B50822019379
:1014B800594B856D1F68C36D2E689A4016420446C5
:1014C8000CD001680868400708D5086820F00400B7
:1014D8000860AA60626D42F00102626501229A40CA
:1014E800164208D021684969090641BFAA60626DA1
:1014F80042F00202626504229A40164208D021682E
:101508000968880741BFAA60626D42F004026265FB
:1015180010229A40164210D02368196809070CD582
:10152800AA601A68500335D51B68190301D4236CC7
:1015380000E0A36C0BB1204698472022E16D8A4059
:10154800164238D023681868C60634D5AA6094F8BD
:101558003520052A1A6825D122F016021A605A6920
:1015680022F080025A61226C0AB9A26C1AB11A6878
:1015780022F008021A603F238B40AB60002384F8F6
:101588003430012384F83530236D0BB12046984759
:1015980003B0F0BD1A68D2055EBF1A6822F00802CF
:1015A8001A60C4E7500328D51B68190332D4636C4A
:1015B8000BB120469847636D002BE9D0636DDA07BD
:1015C80019D50523226884F83530136823F0010300
:1015D80013604FF41653B7FBF3F7019B01339F4297
:1015E800019302D31368DB07F7D4002384F834305F
:1015F800012384F83530E36CC7E71A6812F4807267
:1016080008D1196821F010011960012384F83420E9
:1016180084F83530E36BCBE70800002000232DE980
:10162800F74FD1F80080DFF8B4916A4A38FA03F42A
:1016380002D103B0BDE8F08F4FF0010E0EFA03FEA1
:1016480018EA0E0600F0B4804C6824F01007022F48
:1016580016D14FF00F0C4FEAD30A00EB8A0A03F0B9
:10166800070BDAF820504FEA8B0B0CFA0BFC25EA33
:101678000C0C0D6905FA0BF545EA0C05CAF8205063
:1016880003254FEA430A05FA0AF5ED43D0F800B0FE
:1016980004F0030C0BEA050B0CFA0AFC013F4CEAB8
:1016A8000B0C012FC0F800C011D8876807EA050B9A
:1016B800CF6807FA0AFC4CEA0B078760476827EAF5
:1016C8000E0EC4F300179F4047EA0E074760C7682D
:1016D8003D408F6807FA0AF73D43C560E50067D5C6
:1016E8004FF0000B4FF00F0ECDF804B0D9F844704E
:1016F80003F0030C47F48047C9F84470D9F84470E4
:10170800354D07F480470197019F23F0030707F140
:10171800804707F59C37D7F808A04FEA8C0C0EFADB
:101728000CFEA8422AEA0E0E44D005F58065A842B0
:1017380042D005F58065A84240D005F58065A842ED
:101748003ED005F58065A8423CD005F58065A842E5
:101758003AD005F58065A84238D005F58065A842DD
:1017680036D005F58065A84214BF0925082505FA75
:101778000CF545EA0E05BD60F743156814F4803F83
:101788000CBF3D4035431560556814F4003F0CBF4D
:101798003D4035435560956814F4801F0CBF3D40AB
:1017A80035439560D568A40254BF3D403543D560A4
:1017B80001333BE75D46DAE70125D8E70225D6E79E
:1017C8000325D4E70425D2E70525D0E70625CEE78B
:1017D8000725CCE7003C01400000024000380240E9
:1017E8000369194214BF0120002070470AB18161C2
:1017F80070470904FBE743690B4218BF090481617C
:101808007047000008B5044B5969014202D058617D
:1018180006F022FB08BD00BF003C01400168002221
:101828004B6913F4806310D06FF480634B612023FD
:10183800026380F83D3080F83E20036C80F83C203D
:1018480043F00403036401207047184670472DE9EC
:10185800F843044617469946C1F307488EB22568EF
:10186800B8F1010F0CBF6B69AB6936EA030314BF0B
:101878000120002008B9BDE8F8836B695A0516D520
:101888002B68202243F400732B606FF480636B6134
:101898000023236384F83D2084F83E30226C42F014
:1018A8000402226484F83C300120BDE8F8837B1CE4
:1018B800D5D0FFF793FCA0EB0900874201D3002F96
:1018C800CDD100232022236384F83D2084F83E30C4
:1018D800226C42F02002E4E770B504460D46164635
:1018E80023685B695B0701D5002070BD2046FFF7C0
:1018F80095FFA8B96A1CF3D0FFF770FC801B8542DE
:1019080001D3002DECD100232022236384F83D204D
:1019180084F83E30226C84F83C3042F02002226485
:10192800012070BD70B504460D461646206843690F
:1019380013F0400301D0002070BD4269D2060ED5D5
:101948006FF0100242612022236384F83D2084F85E
:101958003E30226C226484F83C30012070BDFFF7D1
:101968003DFC801BA84201D8002DDFD10023202296
:10197800236384F83D2084F83E30226C42F0200234
:10198800E8E72DE9F843044690461F46089EC1F350
:1019980007498DB22368B9F1010F0CBF5B699B69D8
:1019A80035EA03030CBF01230023434502D000207E
:1019B800BDE8F8837B1CEDD0FFF710FC801B874245
:1019C80001D3002FE6D100232022236384F83D2091
:1019D80084F83E30226C84F83C3042F020022264C5
:1019E8000120BDE8F88370B504460D461646236805
:1019F8005B691B0601D5002070BD2046FFF70EFF6E
:101A0800A8B96A1CF3D0FFF7E9FB801B854201D314
:101A1800002DECD100232022236384F83D2084F894
:101A28003E30226C84F83C3042F0200222640120CF
:101A380070BD00002DE9FF411546026898461368FD
:101A48000B9E43F4807313600F4600960A9B002296
:101A58004FF001110446FFF794FF18B1012004B0BC
:101A6800BDE8F081236807F0FE071F610A9A334634
:101A780016492046FFF7EBFE0028EFD123680390B4
:101A88005A690A9903929B69324603932046039B3D
:101A9800FFF7A9FF40B1236C042B01BF226813682C
:101AA80043F400731360D9E7B8F1010F236802D13A
:101AB800EDB21D61D3E72A0A1A610A993246204617
:101AC800FFF791FF0028E6D12368F1E70200010043
:101AD8002DE9FF419846036816461A680B9D42F4A3
:101AE80080621A601A680F4642F480721A604FF0DA
:101AF800011100950A9B00220446FFF742FF18B126
:101B0800012004B0BDE8F0812368FFB207F0FE02AF
:101B18001A6129492B460A9A2046FFF798FE0028A1
:101B2800EED1236803905A690A9903929B692A4661
:101B380003932046039BFFF756FF40B1236C042B09
:101B480001BF2268136843F400731360D8E7B8F143
:101B5800010F236825D1F6B21E612A460A9920464C
:101B6800FFF741FF02460028E8D1216820460B68AC
:101B780043F480730B6000950A9B4FF00111FFF747
:101B880000FF0028BCD1236847F001071F610A9AAB
:101B98002B4609492046FFF75AFE003018BF01209E
:101BA800AFE7320A1A610A992A462046FFF71BFF57
:101BB8000028C3D12368CEE70200010070B50446AF
:101BC80008B9012070BD90F83D3003F0FF021BB941
:101BD80080F83C2006F0ECFC2423226884F83D3091
:101BE800136823F00103136000F098FC6568414B0B
:101BF8009D424DD8404B9842E3D940492268B0FBFA
:101C0800F1F1536823F03F030B435360136A23F049
:101C18003F03013119431162D169364B21F44F4119
:101C28009D4221F0FF0100F1FF3048D86D00B0FB64
:101C3800F5F00130C0F30B03042B38BF04230B432A
:101C4800D3611168206AE36921F0C00103430B43A3
:101C580013609168E068236921F40341034321F08C
:101C6800FF010B439360D168A069636921F0FF010C
:101C780003430B43D3601368002043F00103136050
:101C88002023206484F83D30206384F83E0070BD32
:101C98001B4B984295D9194E4FF49671B0FBF6F646
:101CA80022687143536823F03F0333434FF47A7635
:101CB8005360136AB1FBF6F123F03F03A9E7A36869
:101CC80053B905EB4503B0FBF3F0431CC3F30B0317
:101CD8006BB143F40043B2E719236B43B0FBF3F055
:101CE800431CC3F30B0313B143F44043A7E7012399
:101CF800A5E700BFA08601007F841E0040420F00B8
:101D0800FF083D002DE9F743044699460F469046E3
:101D18000C9EFFF763FA94F83D300546202B03D05C
:101D2800022003B0BDE8F0830090192301223B494B
:101D38002046FFF726FE0028F2D194F83C30012B0C
:101D4800EED0012384F83C30236820461A68D10776
:101D580058BF1A6839465CBF42F001021A601A6817
:101D680022F400621A60212384F83D30402384F86D
:101D78003E30002323640A9B01956362BDF82C3032
:101D880000966385638D42462385254BE3624B4667
:101D9800FFF750FE00282AD00120C2E7FFF723FEF4
:101DA80040B1236C042B01BF2268136843F400730D
:101DB8001360F1E7636A27681A4612F8011B396154
:101DC8006262628D218D013A92B262857A69481EFB
:101DD80080B2520720850AD548B15A7802333A6151
:101DE8006362638D0239013B9BB221856385238D34
:101DF8002A4631462046002BD0D1FFF76DFD00283A
:101E0800CFD12268136843F400731360202384F849
:101E18003C0084F83D3084F83E0082E70200100060
:101E28000000FFFF2DE9F043044687B099460D46B0
:101E38009046109FFFF7D2F994F83D300646202BC4
:101E480004D00225284607B0BDE8F0830090192386
:101E5800012277492046FFF794FD0028F1D194F834
:101E68003C30012BEDD0012384F83C30236829460F
:101E78001A68D00758BF1A6820465CBF42F00102B2
:101E88001A601A6822F400621A60222384F83D302E
:101E9800402384F83E30002323640E9B019663623E
:101EA800BDF83C3000976385638D42462385614BBE
:101EB800E3624B46FFF70CFE054608B10125C1E772
:101EC800228D236892B902905A6902929A69029205
:101ED800029A1A6842F400721A60202384F83D308E
:101EE800002384F83E3084F83C30ABE7012A2CD13B
:101EF8001A6822F480621A6003905A6903929A69F8
:101F08000392039A1A6842F400721A60DFF8288173
:101F1800238D002BE1D0032B6ED8012B2DD1324617
:101F280039462046FFF7FEFC0028C7D12268636ABD
:101F380012691A70636A01336362238D013B23853A
:101F4800638D013B9BB26385E2E7022A0ED11A68D2
:101F580022F480621A601A6842F400621A600490DF
:101F68005A6904929B690493049BCFE705905A69C8
:101F780005929B690593059BC8E7022B00963B4693
:101F88004FF000024146204619D1FFF7FAFC00281D
:101F980094D123681A6842F400721A601B69626A55
:101FA8001370626A531C6362238D013B2385638D22
:101FB800013B9BB2638523681B695370BAE7FFF73F
:101FC800E0FC024600287FF479AF236820461968B0
:101FD80021F4806119601B69616A0B70636A00965D
:101FE80001336362238D4146013B2385638D013BA9
:101FF8009BB263853B46C8E7324639462046FFF721
:1020080091FC00287FF45AAF2268636A12691A703B
:10201800626A531C6362238D013B2385638D013BF8
:102028009BB263852368596949077FF571AFC3E798
:10203800020010000000FFFF040001002DE9F34139
:10204800044608B901203BE00368DD0710D4236883
:10205800980745D423681A0700F1918023685B0725
:1020680000F1AF80A069002840F00181002027E03E
:10207800AA4B9A6802F00C02042A07D09A6802F068
:102088000C02082A0AD15B68590207D5A34B1B68C2
:102098009A03DCD56368002BD9D1D3E7A04B22790A
:1020A8001A7063687BB1FFF799F806469B4D2B6859
:1020B8009B03CCD4FFF792F8801B6428F7D9032040
:1020C80002B0BDE8F081FFF789F80646934D2B680A
:1020D8009F03BCD5FFF782F8801B6428F7D9EEE789
:1020E8008E4B9A6812F00C0F07D09A6802F00C0217
:1020F800082A16D15B685E0213D4884B1A689507C4
:1021080002D5E268012A9DD11868F82292FAA2F253
:10211800B2FA82F122698A4020F0F8010A431A6073
:1021280098E7E2687F4BDAB101221A60FFF756F8A8
:1021380006467A4D2B6898070CD52968F82393FA38
:10214800A3F3B3FA83F22369934021F0F80213430F
:102158002B607FE7FFF742F8801B0228EAD9AEE739
:102168001A60FFF73BF806466C4D2B6899077FF518
:1021780071AFFFF733F8801B0228F6D99FE7626931
:10218800694B7AB101221A60FFF728F80646634DB9
:102198006B6F9F073FF562AFFFF720F8801B02289F
:1021A800F6D98CE71A60FFF719F806465B4D6B6F96
:1021B80098077FF553AFFFF711F8801B0228F6D96F
:1021C8007DE7564B1A6C12F0805226D101260192F7
:1021D8001A6C42F080521A641B6C03F0805301930E
:1021E800019B524D2B6843F480732B602B68D905F3
:1021F80015D54F4B227A1A70A36803BBFEF7EEFF82
:1022080041F288380746454D2B6F980720D5FEF7D1
:10221800E5FFC01B4045F7D951E70026E1E72B68E9
:1022280043F480732B60FEF7D9FF07462B68DA0565
:10223800DFD4FEF7D3FFC01B0228F7D93FE7FEF72C
:10224800CDFF41F288380746344D2B6F9B0708D5E0
:10225800002E3FF407AF314A136C23F08053136408
:1022680000E7FEF7BBFFC01B4045EED927E72B4D23
:10227800AB6803F00C03082B5ED000232D4E022818
:1022880033603ED1FEF7AAFF07462B68990132D486
:1022980047F6C07797FAA7F74FF44032B7FA87F7AF
:1022A80092FAA2F24FF07061B2FA82F091FAA1F1BB
:1022B800B1FA81F1226AE3691343626A02FA07F705
:1022C800A26A3B435208013A82401343E26A134C24
:1022D80002FA01F10B436B6001233360FEF77EFFC6
:1022E800054623689A013FF5C1AEFEF777FF401B0C
:1022F8006428F6D9E3E6FEF771FFC01B6428C4D949
:10230800DDE6FEF76BFF04462B689B017FF5AEAE5A
:10231800FEF764FF001B6428F6D9D0E600380240B7
:102328000238024000004742800E474200700040D9
:10233800703802406000474201283FF4C1AE686827
:10234800E36900F480029A427FF47CAE226A00F0CE
:102358003F0393427FF476AE626AC0F388139342D8
:102368007FF470AEA26A00F4403393427FF46AAE01
:10237800E36A00F07060C01A18BF0120A0E600BF31
:10238800134908B58B6803F00C03042B03D0082B02
:1023980003D0104808BD104808BD4A684B68496812
:1023A80013F4800314BF0C480A48C1F3881118BFFE
:1023B800002302F03F02A1FB0001FEF73DFD044BA4
:1023C8005B68C3F3014301335B00B0FBF3F008BD66
:1023D800003802400024F40040787D012DE9F041E6
:1023E8000D46044610B90120BDE8F081464B1A6835
:1023F80002F00F028A422FD321688F0734D4C8070E
:1024080047D4414B1A6802F00F0295426BD32268F9
:10241800510771D4130707D53C4A2169936823F4FF
:10242800604343EAC1039360FFF7AAFF374BF022EA
:102438009B6892FAA2F2B2FA82F203F0F003D34058
:10244800334AD35CD840334B1860334B1868FEF7D7
:102458007BFE0020BDE8F081CAB21A701B6803F049
:102468000F039942BFD1C7E7284B11F0040F1EBFD5
:102478009A6842F4E0529A600E0742BF9A6842F4A2
:1024880060429A609A68A06822F0F00202439A605B
:10249800B5E761681D4B01291A681CD112F4003F89
:1024A800A1D09A6841F2883822F003020A439A6060
:1024B800FEF794FE0746154EB368626803F00C03F6
:1024C800B3EB820F9DD0FEF789FEC01B4045F3D9C0
:1024D8000320BDE8F081022902D112F0007FDFE776
:1024E80012F0020FDCE7EAB21A701B6803F00F0360
:1024F8009D427FF478AF8AE70449E0688B6823F44B
:10250800E05303438B6085E7003C024000380240FB
:1025180089B900080800002004000020084B4FF487
:10252800E0529B6892FAA2F2B2FA82F203F4E05304
:10253800D340044AD35C044A1068D840704700BFAF
:102548000038024099B9000808000020084B4FF4F1
:1025580060429B6892FAA2F2B2FA82F203F46043F4
:10256800D340044AD35C044A1068D840704700BF7F
:102578000038024099B900080800002003680020CC
:10258800DA6842F00102DA609A6802F00702062A65
:102598001EBF1A6842F001021A6070477047704700
:1025A80070477047036810B51A69044691070ED53D
:1025B800DA6892070BD56FF002021A6101229B6953
:1025C80002779B0777D0FFF7EAFF0023237723687A
:1025D8001A69500710D5DA6851070DD56FF0040253
:1025E8001A6102229B69227713F4407F204668D043
:1025F800FFF7D5FF0023237723681A6912070FD541
:10260800DA6810070CD56FF008021A610422DB693A
:102618002277990720465AD0FFF7C1FF0023237776
:1026280023681A69D20610D5DA68D0060DD56FF07E
:1026380010021A610822DB69227713F4407F2046D2
:102648004BD0FFF7ACFF0023237723681A69D10723
:1026580008D5DA68D20705D56FF0010220461A615D
:1026680005F0ACFB23681A69100608D5DA6811066C
:1026780005D56FF0800220461A6100F0D4F823686F
:102688001A69520608D5DA68500605D56FF0400277
:1026980020461A61FFF785FF23681A69910622D53B
:1026A800DA6892061FD56FF020022046BDE8104078
:1026B8001A6100F0B7B8FFF771FF2046FFF770FF07
:1026C80083E7FFF76BFF2046FFF76AFF92E7FFF704
:1026D80065FF2046FFF764FFA0E7FFF75FFF20468E
:1026E800FFF75EFFAFE710BD304A0368904212D093
:1026F800B0F1804F0FD0A2F57C4290420BD002F58A
:102708008062904207D002F58062904203D002F5C1
:102718007842904219D14A6823F070031343234A40
:10272800904229D0B0F1804F26D0A2F57C42904249
:1027380022D002F5806290421ED002F5806290425B
:102748001AD002F57842904216D0194A904213D016
:1027580002F5806290420FD002F5806290420BD061
:10276800A2F59832904207D002F58062904203D0D9
:1027780002F58062904203D1CA6823F44073134380
:102788004A6923F08003134303608B68C3620B68B4
:102798008362064B984203D003F58063984201D1C7
:1027A8000B69036301234361704700BF00000140C8
:1027B8000040014010B50446A0B190F83D3003F048
:1027C800FF021BB980F83C2005F04AFF022320686D
:1027D80084F83D30211DFFF787FF0123002084F88E
:1027E8003D3010BD012010BD90F83C3030B5012BB4
:1027F8004FF0020314D0046880F83D306268A36883
:102808000D68496822F0700223F080030B432A43C5
:102818006260A360012380F83D30002380F83C30DB
:10282800184630BD704770470368DA6822F4907222
:10283800DA605A6922F001025A61202380F83A309E
:102848007047000038B504460368C1681A692569ED
:1028580022F440520A431A61A268D9682A4365697A
:10286800C0692A4321F4164121F00C0102430A43AE
:10287800DA605A69A16922F440720A43B0F5004F40
:102888005A61224A24D1934203D002F580629342CE
:102898001BD1FFF75BFE19235843636821685B006F
:1028A8006424B0FBF3F0B0FBF4F504FB1503DB0084
:1028B8003233B3FBF4F303F007025B0002EB0512BB
:1028C80003F4F87313448B6038BDFFF727FEE2E783
:1028D800934202D00E4A934214D1FFF737FE1923D0
:1028E8005843636864229B00B0FBF3F02168B0FB97
:1028F800F2F402FB14031B013233B3FBF2F303EBD4
:102908000413E0E7FFF70AFEE9E700BF0010014003
:1029180000140140F8B504460E4617461D462168C6
:102928000B6836EA030301D10020F8BD6B1CF7D011
:1029380095B923680320DA6822F4D072DA605A69FC
:1029480022F001025A61202384F8393084F83A30A1
:10295800002384F83830F8BDFEF740FCC01B8542E0
:10296800DDD2E6E710B5044640B390F8393003F0FD
:10297800FF021BB980F8382005F08AFE242322685C
:1029880084F83930D368204623F40053D360FFF726
:1029980059FF236800201A6922F490421A615A6983
:1029A80022F02A025A61DA6842F40052DA602023DF
:1029B800E06384F8393084F83A3010BD012010BD46
:1029C8002DE9F0411F4690F839300446202B0D467A
:1029D80090464ED1002949D0002A47D090F8383087
:1029E800012B46D0012380F838300023C36321230C
:1029F80080F83930FEF7F2FB0646A4F82480A4F8E4
:102A08002680E38C9BB26BB93B4632464021204678
:102A1800FFF780FFA8B9202384F8380084F83930FC
:102A2800BDE8F081E38C3246013B9BB2E384A368A6
:102A38008021B3F5805F20463B460ED1FFF76AFF41
:102A480010B10320BDE8F0812B882268C3F3080386
:102A58005360236943B90235D3E7FFF75BFF0028CA
:102A6800EFD123682A785A600135CAE70120BDE80A
:102A7800F0810220BDE8F08138B50446134694F889
:102A88003920202A2AD139B333B394F83820012ABF
:102A980024D00122002584F838202122E384206BE9
:102AA800E56384F839200E4AA3842162C2630D4A83
:102AB800056502640C4AC26422680432FEF7A6FC6B
:102AC8006FF04002236828461A605A6984F8385023
:102AD80042F080025A6138BD012038BD022038BD5D
:102AE800872B0008B52B0008812C0008134690F8A6
:102AF8003A2073B5202A054638D1002934D0002B56
:102B080032D090F83820012A30D00122002480F8F1
:102B180038202222C4638162838580F83A20406B82
:102B2800134A2E68C263134A04650264124AC264D7
:102B38000A46311DFEF76AFC20462B6801941A6884
:102B480001925A6885F838400192019ADA6842F48D
:102B58008072DA605A6942F001025A615A6942F099
:102B680040025A6102B070BD0120FBE70220F9E77C
:102B7800BF2B0008752C0008812C0008704708B589
:102B88000368826B1B6813F480730AD1D3841368BB
:102B98005A6922F080025A61DA6842F04002DA602B
:102BA80008BD1046FFF7EAFF08BD704708B5806BFF
:102BB800FFF7FBFF08BD08B50368826B1B6813F4B9
:102BC800807310D1D3851368D96821F48071D960D6
:102BD800596921F001015961596921F04001596190
:102BE800202382F83A30104605F00CF908BD90F819
:102BF8003A3010B5222B36D183680169B3F5805F6E
:102C08000268836A23D15268E9B9C2F3080223F83B
:102C1800022B8362C48D013CA4B2C4858CB90368BD
:102C2800DA6822F02002DA60DA6822F48072DA6068
:102C38005A6922F001025A61202380F83A3005F0DF
:102C4800E1F8002010BDD2B223F8012BE1E721B949
:102C5800591C526881621A70DCE75268591C8162FB
:102C680002F07F02F7E7022010BD704708B5806BBD
:102C7800FFF7FBFF08BD7047816B08B50B685A6901
:102C880091F8390021280AD1120608D50022CA84F1
:102C9800DA6822F0C002DA60202281F839205B6904
:102CA80091F83A20222A06D15B0604D5002308466B
:102CB800CB85FFF7B9FDCB6B084643F01003CB6318
:102CC800FFF7D9FF08BD0000036870B51A6804460D
:102CD8001607D9685D6907D196065AD58D0658D565
:102CE800BDE87040FFF783BF15F0010502D111F46C
:102CF800907F4ED0D30705D5CE0542BFE36B43F096
:102D08000103E363500704D51DB1E36B43F00203ED
:102D1800E363930704D51DB1E36B43F00403E36356
:102D2800160704D51DB1E36B43F00803E363E36BB7
:102D3800002B66D0950604D5880602D52046FFF7F5
:102D480056FF236820465D69E26B110702D415F02F
:102D580040051AD0FFF768FD23685A69520610D556
:102D68005A69606B22F040025A6150B1254B0365E5
:102D7800FEF787FB002844D0606BBDE87040036D08
:102D880018472046FFF777FF70BDFFF774FFE5632C
:102D980070BD160627D50D0625D594F83920212AA9
:102DA8002FD1A268B2F5805F226A17D11188C1F3CA
:102DB80008015960216979B902322262E28C013A2C
:102DC80092B2E284EAB9DA6822F08002DA60DA685C
:102DD80042F04002DA6070BD0132EEE7511C216218
:102DE80012785A60EAE750060BD54A0609D5DA6820
:102DF800204622F04002DA60202384F83930FFF7B9
:102E0800BDFE70BD112E000808B50023806BC38578
:102E1800C384FFF730FF08BD014B1870704700BF2F
:102E280030020020014B1878704700BF30020020A4
:102E380010B50446087801F061FA206010BD38B575
:102E4800044608780D4601F059FA2060687801F0C8
:102E580055FA01462068FDF751FE2060A87801F078
:102E68004DFA01462068FDF749FE2060E87801F038
:102E780045FA01462068FDF741FE206038BD38B5A7
:102E8800044608780D4601F0C9FA2060687801F018
:102E9800C5FA01462068FDF731FE2060A87801F0E8
:102EA80075FA01462068FDF729FE206038BD00004C
:102EB8000138122838D8DFE800F00A3737372237C8
:102EC800370E1215191C1F25282B2E3134001749CF
:102ED8001748FFF7ADBF17491748FFF7B0BF1749A5
:102EE8001748FAE717491848FFF7C9BF174918489C
:102EF800FAE718491848F7E718491948F4E719494B
:102F08001948E6E719491A48E7E71A491A48E4E769
:102F18001A491B48E8E71B491B48E5E71B491C48B9
:102F2800E2E71C491C48DFE7704700BF1A09002088
:102F3800F80100201B0900200C0200201F090020B6
:102F48001002002023090020FC010020260900208F
:102F58000002002029090020040200202C0900207A
:102F6800080200202F090020140200203009002048
:102F780028020020340900202C02002038090020F3
:102F8800180200203B0900201C0200203E090020F6
:102F98002002002041090020240200200023DAB288
:102FA800815C01330029FAD1104670472DE9F047BA
:102FB8004FF0100A4FF020099EB001AF80460D4631
:102FC800144600215246384605AE05F07CFD4A46B7
:102FD8000021304605F077FD4FF48053ADF83430CA
:102FE8004FF40063ADF836304FF40053ADF8383085
:102FF8004FF48043ADF83C304FF40043ADF83E3019
:103008000423ADF840300823ADF842304023ADF832
:1030180048308023ADF846A0ADF84490ADF84A306A
:10302800B8F1000F02D0404600F01BFA00224FF41E
:1030380078413B48FEF7DAFB0022FC213948FEF7CD
:10304800D5FB002D67D12A464FF400613448FEF7BE
:10305800CDFB0FAB93E8030016AB87E8030093E8BA
:103068000300012286E803004FF400512C48FEF7C4
:10307800BDFB14F0010218BF01224FF4804128481B
:10308800FEF7B4FB14F0020218BF01224FF400410E
:103098002348FEF7ABFB14F0040218BF01220421F9
:1030A8002048FEF7A3FB14F0080218BF01220821EC
:1030B8001C48FEF79BFB14F0100218BF01222021C8
:1030C8001848FEF793FB14F0200218BF01221021C4
:1030D8001448FEF78BFB14F0400218BF0122402170
:1030E8001048FEF783FB23064CBF012200228021F3
:1030F8000C48FEF77BFB00224FF400510848FEF70E
:1031080075FB55B901224FF4006105481EB0BDE8B2
:10311800F047FEF76BBB012296E70022F3E700BFFA
:10312800000C024000180240002138B5AF4C0C22B8
:103138000846FFF73BFFA07901F0E0F8AC4BAD4D36
:103148001860E07901F0DAF801462868FDF7D6FC46
:103158002860207A01F0D2F801462868FDF7CEFCF5
:103168002860607A01F0CAF801462868FDF7C6FCB5
:103178002860A07A01F0C2F801462868FDF7BEFC75
:103188002860E07A01F0BAF89B4D01462868FDF7FF
:10319800B5FC2860207B01F0B1F801462868FDF7EE
:1031A800ADFC2860607B01F0A9F801462868FDF7AE
:1031B800A5FC2860A07B01F0A1F801462868FDF76E
:1031C8009DFC2860E07B01F029F98C4D01462868B8
:1031D800FDF794FC2860207C01F020F9014628685E
:1031E800FDF78CFC2860607C01F0D0F80146286867
:1031F800FDF784FC2860A07C01F010F9804D0146A1
:103208002868FDF77BFC2860E07C01F007F901469F
:103218002868FDF773FC2860207D01F0B7F80146A7
:103228002868FDF76BFC2860607D01F0F7F8754DA4
:1032380001462868FDF762FC2860A07D01F0EEF8E1
:1032480001462868FDF75AFC2860E07D01F09EF8E9
:1032580001462868FDF752FC2860207E01F0DEF860
:10326800694D01462868FDF749FC2860607E01F039
:10327800D5F801462868FDF741FC2860A07E01F0DA
:1032880085F801462868FDF739FC2860E07E01F0E2
:1032980035F85E4B5E4D1860207F01F02FF801462F
:1032A8002868FDF72BFC2860607F01F027F80146AD
:1032B8002868FDF723FC2860A07F01F01FF801466D
:1032C8002868FDF71BFC2860E07F01F017F801462D
:1032D8002868FDF713FC286094F8200001F00EF828
:1032E8004C4D01462868FDF709FC286094F8210038
:1032F80001F004F801462868FDF700FC286094F8FE
:10330800220000F0FBFF01462868FDF7F7FB286064
:1033180094F8230000F0F2FF01462868FDF7EEFB61
:10332800286094F8240001F079F83B4D014628689C
:10333800FDF7E4FB286094F8250001F06FF80146DA
:103348002868FDF7DBFB286094F8260001F01EF8DA
:1033580001462868FDF7D2FB286094F8270001F0A1
:103368005DF82E4D01462868FDF7C8FB286094F8E3
:10337800280001F053F801462868FDF7BFFB2860D4
:1033880094F8290001F002F801462868FDF7B6FB19
:10339800286094F82A0001F041F8214D0146286878
:1033A800FDF7ACFB286094F82B0001F037F80146D4
:1033B8002868FDF7A3FB286094F82C0000F0E6FFCE
:1033C80001462868FDF79AFB286094F82D0001F063
:1033D80025F8144D01462868FDF790FB286094F8FD
:1033E8002E0001F01BF801461EE000BF1409002062
:1033F800F80100200C02002010020020FC0100202F
:10340800000200200402002008020020140200200C
:10341800280200202C020020180200201C02002094
:1034280020020020240200202868FDF767FB28609E
:1034380094F82F0000F0AAFF01462868FDF75EFB0C
:10344800286038BD00210F220846FFF7AFBD0021D4
:103458000C220846FFF7AABD002101220846FFF703
:10346800A5BD002101280CBF8022C0220846FFF715
:103478009DBD00002DE9F04F10252024A1B00DF1CD
:103488000C0A904607462A468946504600210DF107
:103498001C0B05F018FB22460021584605F013FBCB
:1034A8004FF48053ADF83C304FF40063ADF83E3034
:1034B8004FF40053ADF840304FF48043ADF844303A
:1034C8004FF40043ADF846300423ADF848300823E4
:1034D800ADF84A304023ADF8503080234046ADF86F
:1034E8004E50ADF84C40ADF85230FFF757FD464608
:1034F800504D514C0190A6EB0803019ADBB29A4259
:1035080002D821B0BDE8F08F002F40F08780002757
:1035180000224FF478412846FEF768F90022FC2182
:103528002046FEF763F9B9F1000F7ED14A464FF401
:1035380000612846FEF75AF911AB93E8030018AB6F
:103548008AE8030093E8030001228BE803004FF4A4
:1035580000512846FEF74AF916F8012B4FF480412E
:1035680012F0010218BF01222846FEF73FF916F8AB
:10357800012C4FF4004112F0020218BF0122284624
:10358800FEF734F916F8012C042112F0040218BFD2
:1035980001222046FEF72AF916F8012C082112F01C
:1035A800080218BF01222046FEF720F916F8012C60
:1035B800202112F0100218BF01222046FEF716F94A
:1035C80016F8012C102112F0200218BF0122204603
:1035D800FEF70CF916F8012C402112F0400218BF32
:1035E80001222046FEF702F916F9013C8021002B42
:1035F800B4BF012200222046FEF7F8F800224FF45B
:1036080000512846FEF7F2F8B9F1000F0FD1012258
:103618004FF400612846FEF7E9F86CE73846FFF7F3
:1036280020FF022F3FF473AF72E701227FE70022E9
:10363800EEE700BF000C024000180240014B18786A
:10364800704700BF320200201FB510240021224617
:10365800684605F038FAFFF7FAFEFFF7FDFE0C4A58
:1036680001210020FFF706FF224601210020FFF775
:103678009DFC0849684605F0E5FF6A4601210220DD
:10368800FFF7F8FE0022044B1A7004B010BD00BF0B
:103698000CB800081CB80008320200201FB510241E
:1036A80000212246684605F00EFAFFF7D0FEFFF724
:1036B800D3FE0F4A01210020FFF7DCFE224601213C
:1036C8000020FFF773FC0B4B1868FCF7E5FE0B4670
:1036D80002460949684605F091FF6A460121022021
:1036E800FFF7C8FE0122054B1A7004B010BD00BFD9
:1036F800E1B70008F8010020F0B700083202002006
:103708001FB5102400212246684605F0DCF9FFF7B2
:103718009EFEFFF7A1FE112201210020FFF746FCC3
:103728000E4A01210020FFF7A5FE224601210020B4
:10373800FFF73CFC0A4B1868FCF7AEFE0B46024646
:103748000849684605F05AFF6A4601210220FFF73A
:1037580091FE0222044B1A7004B010BD28B800086C
:103768000C020020F0B70008320200201FB510221A
:103778000021684605F0A7F9FFF769FEFFF76CFE20
:10378800112201210020FFF711FC0D4A0121002020
:10379800FFF770FE0B4B1868FCF77EFE0B460246DF
:1037A8000949684605F02AFF6A4601210220FFF709
:1037B80061FE0322054B1A7005B05DF804FB00BFDB
:1037C80000B80008FC010020F0B700083202002011
:1037D8001FB510220021684605F075F9FFF737FE7E
:1037E800FFF73AFE112201210020FFF7DFFB0A4A0A
:1037F80001210020FFF73EFE0849684605F022FF38
:103808006A4601210220FFF735FE0422044B1A7094
:1038180005B05DF804FB00BF52B800081CB80008EA
:10382800320200201FB5102400212246684605F008
:103838004AF9FFF70CFEFFF70FFE0F4A012100209F
:10384800FFF718FE224601210020FFF7AFFB0B4BC4
:103858001868FCF721FE0B4602460949684605F040
:10386800CDFE6A4601210220FFF704FE0522054B22
:103878001A7004B010BD00BF37B800081402002049
:10388800F0B70008320200201FB51024002122469C
:10389800684605F018F9FFF7DAFDFFF7DDFD11229C
:1038A80001210020FFF782FB0E4A01210020FFF7CB
:1038B800E1FD224601210020FFF778FB0A4B18683A
:1038C800FCF7EAFD0B4602460849684605F096FEF5
:1038D8006A4601210220FFF7CDFD0622044B1A702B
:1038E80004B010BD5EB8000828020020F0B7000838
:1038F800320200201FB510220021684605F0E3F8C7
:10390800FFF7A5FDFFF7A8FD112201210020FFF711
:103918004DFB0D4A01210020FFF7ACFD0B4B186849
:10392800FCF7BAFD0B4602460949684605F066FEF3
:103938006A4601210220FFF79DFD0722054B1A70F8
:1039480005B05DF804FB00BF46B800081802002067
:10395800F0B70008320200202DE9F0410C46164667
:1039680086B010220021804602A805F0ACF8FFF7C7
:1039780069FD21683046FDF7C1F8194F20603946C6
:103988000546FDF72FFA18B1276006B0BDE8F081AB
:10399800002728463946FDF707FA0028F4D12846BB
:1039A800FCF77AFD02460B4602A80E4905F026FEF2
:1039B8002068FCF771FD044630460D46FCF76CFDA7
:1039C8002B46CDE900012246074805F0E5FC02AA8E
:1039D80001210220FFF74EFD044B83F80080D4E755
:1039E8000000F041F0B7000869B700083202002073
:1039F800F0B50C46154685B01022002107466846EA
:103A080005F061F8FFF71EFD21682846FDF776F8F6
:103A1800104E206031460546FDF7E4F910B12660E6
:103A280005B0F0BD002628463146FDF7BDF900284F
:103A3800F5D12846FCF730FD0B4602460649684694
:103A480005F0DCFD6A4601210220FFF713FD034B58
:103A58001F70E5E70000F042F0B7000832020020CE
:103A6800F0B50C46154685B0102200210746684679
:103A780005F029F8FFF7E6FC21682846FDF73EF82F
:103A8800104E206031460546FDF7ACF910B12660AE
:103A980005B0F0BD002628463146FDF785F9002817
:103AA800F5D12846FCF7F8FC0B460246064968465D
:103AB80005F0A4FD6A4601210220FFF7DBFC034B59
:103AC8001F70E5E70000B442F0B70008320200209A
:103AD80030B5044685B010220D466846002104F032
:103AE800F2FFFFF7B4FCFFF7B7FC082C01D00E2C4F
:103AF8001BD1154A01210020FFF7BCFC102201212F
:103B08000020FFF753FA2868FCF7C6FC0B4602466C
:103B18000E49684605F072FD6A4601210220FFF74A
:103B2800A9FC0B4B1C7005B030BD092C01D00F2C23
:103B3800E9D1112201210020FFF738FA054A0121B5
:103B48000020FFF797FCDEE7C1B70008F0B70008D0
:103B580032020020D1B7000830B5044685B01022E3
:103B68000D466846002104F0AEFFFFF770FCFFF732
:103B780073FC0A2C01D0102C1BD1204A01210020F3
:103B8800FFF778FC102201210020FFF70FFA2868C0
:103B9800FCF782FC0B4602461949684605F02EFDE3
:103BA8006A4601210220FFF765FC164B1C7005B020
:103BB80030BD0B2C01D0112C06D11122012100207F
:103BC800FFF7F4F9104AD9E70C2C01D0122C06D1D2
:103BD800112201210020FFF7E9F90C4ACEE70D2C4C
:103BE80001D0132CD3D1112201210020FFF7DEF9D7
:103BF800074A01210020FFF73DFCC8E784B7000809
:103C0800F0B700083202002094B70008A3B70008F4
:103C1800B2B7000838B5AD4D04462B789BB968B9E2
:103C2800FFF71AFC2046AA4A0121FFF723FCBDE84A
:103C38003840A84A01210220FFF71CBCFFF704FD09
:103C480001232B7038BD022803D1BDE83840FFF7A7
:103C5800FBBCA14B1D782846FFF72AF9212D00F25D
:103C68007081DFE815F022003800450058002F0069
:103C7800620071007E00850093009E00AC00B900D0
:103C8800C600CE00DD00E500F000FD000A011201CB
:103C98002D016F018701B301DD01080233024802DB
:103CA80061027A02A502EA021503042C03D1BDE8D9
:103CB8003840FFF78DBD052C40F04381BDE8384002
:103CC800FFF7ECBC032CC0D0052C40F03A81BDE8CE
:103CD8003840FFF7A7BD042C03D1BDE83840FFF7F3
:103CE8000FBD052C40F02D8100227C49142027E0CF
:103CF800042C03D1BDE83840FFF738BD032CDDD0D4
:103D0800052C05D108207649BDE83840FFF7E0BE0C
:103D1800012C9AD038BD032CDFD0052CF8D10A200D
:103D28007049BDE83840FFF717BF042C03D1BDE840
:103D38003840FFF7A9BD052CEAD100221B206A49AB
:103D4800BDE83840FFF708BE042C03D1BDE8384071
:103D5800FFF7D0BD032CBAD0052CD9D163490E206A
:103D6800D2E7032CE3D0052CD2D161491020D8E743
:103D7800042C02D15F490920C6E7052C03D1002293
:103D88005749152009E0012C98D038BD032CB9D02B
:103D9800052CF8D1002216205649BDE83840FFF717
:103DA80027BE042C02D154490B20BAE7052CEAD1CE
:103DB80000224C491720BDE83840FFF751BE042CBB
:103DC80002D14E490C20ACE7032CA8D0052CDAD13F
:103DD800002249491820EEE7042C02D148490D2059
:103DE8009FE7032CDFD0052CCDD1002243491920B1
:103DF800E1E7032CE5D0052CC5D1002240491A2063
:103E0800D9E7042C02D13F490F207DE7052C03D1C7
:103E1800002236491C20C0E7012C3FF458AF38BDBA
:103E2800032C9BD0052CF7D1002236491D20B4E77E
:103E3800042C02D13449112073E7052CECD100225F
:103E48002B491E20B7E7042C02D13049122068E71D
:103E5800032C8AD0052CDFD100222B491F20AAE78A
:103E6800042C02D12A4913205BE7032CE2D0052C4D
:103E7800D2D10022254920209DE7032CE5D0052C2E
:103E8800CAD100222249212095E7032C02D14FF004
:103E98007C522AE7042C02D14FF03F4225E7052C3B
:103EA8007FF471AF0D4C002221461420FFF754FD1A
:103EB8000121206800F002FC0122164B1A7038BD5F
:103EC800032C29D14FF07C525AE700BF330200205F
:103ED80048B7000858B7000832020020F80100204F
:103EE8000C020020FC0100201402002028020020FF
:103EF8001802002010020020000200200402002006
:103F0800080200202C0200201C02002020020020B1
:103F18002402002031020020042C02D14FF03F423D
:103F28002EE7052C0AD1A84C0221206800F0F6FBE8
:103F3800002221461520FFF75BFDBDE7012C3FF469
:103F4800E1AE38BD032C02D14FF07C5223E7042C9C
:103F580002D14FF03F421EE7052C08D19B4C0321AC
:103F6800206800F0DBFB002221461620E3E7012C45
:103F7800E7D1FFE6032C0CD1954C96492068FCF755
:103F88001DFF18B14FF07E52214613E74FF07C52C7
:103F9800FAE7042C0AD18E4C8E492068FCF70EFFF4
:103FA80008B18D4AF0E74FF03F42EDE7052C0AD102
:103FB800874C0421206800F02DFC002221461720A0
:103FC800FFF74EFD78E7012CBBD1A8E6032C0CD1F6
:103FD800824C80492068FCF7F1FE18B14FF07E5200
:103FE8002146F7E64FF07C52FAE7042C0AD17B4CC5
:103FF80078492068FCF7E2FE08B1774AF0E74FF00D
:104008003F42EDE7052C08D1744D2146286800F0A1
:1040180001FC002229461820D2E7012C91D1C2E6E2
:10402800032C0CD16E4C6B492068FCF7C7FE18B105
:104038004FF07E522146DAE64FF07C52FAE7042C24
:104048000AD1674C63492068FCF7B8FE08B1624A98
:10405800F0E74FF03F42EDE7052C08D1604C062110
:10406800206800F0D7FB002221461920A8E7012C80
:104078007FF467AFA5E6032C0CD15A4C554920684C
:10408800FCF79CFE18B14FF07E522146B7E64FF080
:104098007C52FAE7042C0AD1524C4E492068FCF7AE
:1040A8008DFE08B14C4AF0E74FF03F42EDE7052C92
:1040B80008D14C4C0721206800F0ACFB00222146B7
:1040C8001A207DE7012C7FF43CAF87E6032C02D150
:1040D8004FF07C5232E6042C02D14FF03F422DE6DD
:1040E800052C7FF499AE404C002221461B20FFF797
:1040F80033FC0821DDE6032C02D14FF07C5288E620
:10410800042C02D14FF03F4283E6052C08D1374CEE
:104118000921206800F002FB002221461C200AE742
:10412800012C7FF40EAF19E6032C02D14FF07C521C
:104138007BE6042C02D14FF03F4276E6052C08D1ED
:104148002B4C0A21206800F0E9FA002221461D20A4
:10415800F1E6012C7FF4F5AE55E6032C0CD1254C85
:104168001C492068FCF72AFE18B14FF07E52214600
:1041780067E64FF07C52FAE7042C0AD11D4C15492A
:104188002068FCF71BFE08B1134AF0E74FF03F42E6
:10419800EDE7052C08D1174C0B21206800F03AFBFD
:1041A800002221461E200BE7012C7FF4CAAEDCE575
:1041B800032C26D1104C07492068FCF7FFFDE8B115
:1041C8004FF07E52214649E60C02002010020020E2
:1041D800FC01002000007042000080BF00020020A7
:1041E80004020020080200201402002028020020F7
:1041F8002C020020180200201C0200204FF07C52E4
:10420800E0E7042C0AD1384C38492068FCF7D6FD81
:1042180008B1374AD6E74FF03F42D3E7052C08D11B
:10422800314C0C21206800F0F5FA002221461F20AD
:10423800C6E6012C7FF485AEFCE5032C0CD12D4C91
:104248002A492068FCF7BAFD18B14FF07E52214682
:1042580011E64FF07C52FAE7042C0AD1254C234989
:104268002068FCF7ABFD08B1214AF0E74FF03F4268
:10427800EDE7052C08D11F4C0D21206800F0CAFA83
:104288000022214620209BE6012C7FF45AAEDCE573
:10429800032C0CD1184C15492068FCF78FFD18B178
:1042A8004FF07E522146EEE54FF07C52FAE7042C9F
:1042B8000AD1114C0D492068FCF780FD08B10C4A61
:1042C800F0E74FF03F42EDE7052C08D10A4C0E21EC
:1042D800206800F09FFA00222146212070E6012C78
:1042E8007FF42FAEBEE500BF1C0200200000704224
:1042F800000080BF20020020240200202DE9F047A2
:10430800A8B1C0434FF0834500F03F044FF0824608
:1043180000204FF081474FF080484FF07E594FF012
:104328007C5A34B90021FCF7E9FBBDE8F08700208E
:10433800F8E7E10705D5514604F0FE04FCF7DEFB7B
:10434800EFE7A20703D504F0FD044946F6E7630743
:1043580003D504F0FB044146F0E7210703D504F038
:10436800F7043946EAE7E20603D504F0EF043146DC
:10437800E4E7A30603D504F0DF042946DEE7024993
:10438800FCF7BCFBCEE700BF0000FC412DE9F84F6D
:1043980000F03F044FF07C5500204FF07E564FF060
:1043A80080474FF081484FF082494FF0834ADFF849
:1043B80068B03F2C03D15946FCF7A0FB0024A106A6
:1043C80005D5514604F01F04FCF798FBF1E7E20617
:1043D80003D504F02F044946F6E7230703D504F074
:1043E80037044146F0E7610703D504F03B0439463A
:1043F800EAE7A20703D504F03D043146E4E7E30702
:1044080003D504F03E042946DEE7002CD1D1002173
:10441800FCF774FBBDE8F88F0000FC41C0432DE9B0
:10442800F84300F01F044FF0834500204FF0824608
:104438004FF081474FF080484FF07E5924B9002152
:10444800FCF75CFBBDE8F883E20705D5494604F0B4
:104458001E04FCF753FBF1E7A30703D504F01D0482
:104468004146F6E7610703D504F01B043946F0E737
:10447800220703D504F017043146EAE7E30603D51B
:1044880004F00F042946E4E714F01E0F14BF024994
:104498000249FCF733FBD2E70000F8410000FC4179
:1044A8002DE9F74F83463F2400254FF083464FF010
:1044B80082474FF081484FF080494FF07E5A294695
:1044C8005846FCF767FC0190002853D12B49584601
:1044D800FCF760FC019A60B931465846FCF778FC55
:1044E80050B158463146FCF707FB04F01F048346D9
:1044F800E5E71446AB46E2E739465846FCF768FC60
:1045080038B158463946FCF7F7FA04F02F048346C9
:10451800D5E741465846FCF75BFC38B1584641465A
:10452800FCF7EAFA04F037048346C8E749465846D8
:10453800FCF74EFC38B158464946FCF7DDFA04F062
:104548003B048346BBE751465846FCF741FC38B16B
:1045580058465146FCF7D0FA04F03D048346AEE7CE
:104568004FF07C515846FCF733FC0028A7D004F0E4
:104578003E04BFE7204603B0BDE8F08F0000FC41D1
:104588002DE9F84F0546002400264FF083474FF0E9
:1045980082484FF081494FF0804A4FF07E5B3146A8
:1045A8002846FCF7F7FB002858D12E492846FCF787
:1045B800F1FB60B939462846FCF70AFC50B1284699
:1045C8003946FCF799FA44F020040546E7E73F240A
:1045D8003546E4E741462846FCF7FAFB38B1284659
:1045E8004146FCF789FA44F010040546D7E74946E6
:1045F8002846FCF7EDFB38B128464946FCF77CFA1B
:1046080044F008040546CAE751462846FCF7E0FB93
:1046180038B128465146FCF76FFA44F004040546C1
:10462800BDE759462846FCF7D3FB38B1284659461A
:10463800FCF762FA44F002040546B0E74FF07C51FB
:104648002846FCF7C5FB0028A9D028464FF07C5126
:10465800FCF752FA44F001040546A0E72046BDE8FD
:10466800F88F00BF0000FC4103461F202BB31F2B0F
:1046780006D00F2B06D9103BDBB200F00F00F5E790
:1046880000207047072B04D9083BDBB200F0170065
:10469800ECE7032B04D9043BDBB200F01B00E5E791
:1046A800012B89BF023B03F1FF33DBB200F01D0091
:1046B8009CBFDBB200F01E00D8E770471FB500238F
:1046C80002938DF80C30BE238DF8043004238DF846
:1046D80005108DF80630FFF7E3FE3F238DF807003D
:1046E80006210DF105008DF808308DF809308DF898
:1046F8000A30EB2403F007FF074A8DF80B008DF80A
:104708000C4001AB03CB1472106051600120FEF71E
:1047180083FB04B010BD00BF410200201FB5002379
:10472800019302938DF80C30BE238DF804300423D6
:104738008DF80510334904468DF80630FCF752FB16
:1047480018B303232F4920468DF807308DF8083019
:104758008DF80930FCF7D0F9FFF7A2FE8DF80A00B2
:1047680006210DF1050003F0CEFEEB24264A8DF854
:104778000B008DF80C4001AB03CB14721060516034
:104788000120FEF749FB04B010BD20492046FCF784
:1047980029FBA0B11D492046FCF7AEF90446FFF7F6
:1047A8007FFE032320468DF807308DF80830FFF789
:1047B80077FE3F238DF809008DF80A30D0E71449B9
:1047C8002046FCF70FFB70B10323114920468DF8F2
:1047D8000730FCF791F9FFF763FE3F238DF80800D7
:1047E8008DF80930E8E700212046FCF7F1FA0028A7
:1047F800B6D02046FFF754FE3F238DF807008DF80A
:104808000830EDE70000B442410200200000704289
:104818000000F0411FB50023019302938DF80C307E
:10482800BE238DF8043004238DF80510274904466B
:104838008DF80630FCF7D6FA08B301232349204641
:104848008DF807308DF80830FCF756F9FFF798FE19
:104858008DF8090006210DF1050003F054FEEB2444
:104868001B4A8DF80B008DF80C4001AB03CB14727A
:10487800106051600120FEF7CFFA04B010BD154951
:104888002046FCF7A5FA70B10123124920468DF89D
:104898000730FCF731F9FCF7AFFAC0B2FFF7E4FED6
:1048A8008DF80800D6E700212046FCF791FA002889
:1048B800D0D02046FCF7A0FAC0B2FFF7D5FE1F23E0
:1048C8008DF807008DF80830C4E700BF000070427B
:1048D800410200200000F041F8B50646002949D001
:1048E80001294AD002294BD003294CD0042914BFEE
:1048F8004FF480654FF480450624244F16F02002BB
:1049080018BF01224FF400713846FCF76FFF0122EF
:104918004FF480711D48FCF769FF0120FCF764FC27
:1049280000224FF480711948FCF760FF013C012018
:104938007600FCF759FC14F0FF04F6B2DED12246EB
:104948004FF480711148FCF751FF22464FF4007173
:104958000E48FCF74BFF294601220C48FCF746FF9E
:104968000120FCF741FC22462946BDE8F8400748EB
:10497800FCF73CBF4FF48065BEE74FF40065BBE72A
:104988004FF48055B8E74FF40055B5E700100240E2
:104998002DE9F0410546884600294ED001294FD01F
:1049A80002294FD003294FD004290CBF4FF40077B8
:1049B80000270624254E15F0200218BF01224FF4C7
:1049C80000513046FCF712FF01224FF48051304667
:1049D800FCF70CFF0120FCF707FC00224FF4805184
:1049E8003046FCF703FF013C01206D00FCF7FCFB9F
:1049F80014F0FF04EDB2DED122464FF48051134883
:104A0800FCF7F4FE114D124B2246B8F1000F18BF07
:104A18001D464FF400512846FCF7E8FE39460122AE
:104A28002846FCF7E3FE0120FCF7DEFB2246394668
:104A38002846BDE8F041FCF7D9BE4FF48047B8E7F7
:104A48004027B6E78027B4E72027B2E700180240DE
:104A58000004024070B500224FF400410546274883
:104A6800FCF7C4FE00224FF480412448FCF7BEFE48
:104A780000224FF400512148FCF7B8FE08241F4ECD
:104A88002B064CBF012200224FF480413046FCF730
:104A9800ADFE01224FF400511848FCF7A7FE012093
:104AA800FCF7A2FB00224FF400511448FCF79EFECD
:104AB800013C01206D00FCF797FB14F0FF04EDB2F8
:104AC800DED101224FF400410C48FCF78FFE012093
:104AD800FCF78AFB22464FF400410848FCF786FEA3
:104AE80022464FF480410548FCF780FE2246BDE887
:104AF80070404FF400510148FCF778BE00140240A2
:104B080070B500224FF4007105462448FCF76EFE8C
:104B1800002280212248FCF769FE0022402120481B
:104B2800FCF764FE08241E4E2B064CBF012200220F
:104B380080213046FCF75AFE012240211848FCF734
:104B480055FE0120FCF750FB002240211448FCF7D9
:104B58004DFE013C01206D00FCF746FB14F0FF04FC
:104B6800EDB2E1D101224FF400710C48FCF73EFE92
:104B78000120FCF739FB22464FF400710748FCF787
:104B880035FE224680210648FCF730FE2246BDE865
:104B9800704040210248FCF729BE00BF00180240BF
:104BA800000C024038B504460D4610F0100218BF3C
:104BB800012210212248FCF719FE14F0080218BF40
:104BC800012280211F48FCF711FE14F0040218BFCF
:104BD800012240211B48FCF709FE14F0020218BF0D
:104BE800012220211748FCF701FE14F0010218BF2A
:104BF800012210211348FCF7F9FD8DB9012220216B
:104C08000F48FCF7F3FD0120FCF7EEFA2A462021B5
:104C18000B48FCF7EBFDBDE838400120FCF7E4BA8F
:104C2800012D0BD12A4629460748FCF7DFFD284607
:104C3800FCF7DAFA002229460348EAE738BD00BF44
:104C480000080240000002400004024038B5044653
:104C58000D4610F0100218BF012202212348FCF76C
:104C6800C5FD14F0080218BF012201211F48FCF7F6
:104C7800BDFD14F0040218BF01224FF480511C48F6
:104C8800FCF7B4FD14F0020218BF01224FF40061D2
:104C98001748FCF7ABFD14F0010218BF01224FF4CE
:104CA80080611348FCF7A2FD8DB9012204210F4849
:104CB800FCF79CFD0120FCF797FA2A4604210B48D3
:104CC800FCF794FDBDE838400120FCF78DBA012DB2
:104CD8000AD12A4608210548FCF788FD2846FCF732
:104CE80083FA00220821EAE738BD00BF000C024021
:104CF800000802402DE9F047164E04464021304690
:104D0800FCF76EFD144D814602212846FCF768FD2C
:104D1800802107463046FCF763FD04218246284679
:104D2800FCF75EFD4FF4807180463046FCF758FD75
:104D3800082106462846FCF753FD2670E07084F8E3
:104D480001A084F8029084F8048067712046BDE8C9
:104D5800F08700BF001402400008024007B502AB0C
:104D680003E903009DF8023013B19DF8053063BBD9
:104D7800002204211F48FCF739FD012208211D48A3
:104D8800FCF734FD9DF8013013B19DF804301BBBCE
:104D9800002210211748FCF729FD0122202115487F
:104DA800FCF724FD9DF8003013B19DF80330D3B90A
:104DB800002201210F48FCF719FD012202210D48AC
:104DC80003B05DF804EBFCF711BD0122042109488A
:104DD800FCF70CFD0022D1E7012210210548FCF761
:104DE80005FD0022DAE7012202481146FCF7FEFC25
:104DF8000022E3E7001002400A4601460148FDF799
:104E08003BBE00BF0C0E002084B038B504AC84E86B
:104E18000F00149C04ABE21C14A953F8040B8B423A
:104E280042F8040BF9D1A178601CCD1C0231C9B23B
:104E380003F069FBEB226055A378204623441A71DE
:104E4800A1780531C9B2FFF7D7FFBDE8384004B0F3
:104E58007047000084B070B59AB01EAC84E80F00AB
:104E68006422002101A89DF8B8502EAE03F02BFE55
:104E78001EAA01AB1C4610685168083203C4B2422E
:104E88002346F7D13F2D00F2E680DFE805F0202722
:104E98002A2D303336393C3F4245484B4E51545702
:104EA8005A5D606366696C6F7275787B7E818487F2
:104EB8008A8D909396999C9FA2A5A8ABAEB1B4B7E2
:104EC800BABDC0C3C6C9CCCFD2D5D8DBDEE19DF808
:104ED80078001AB0BDE8704004B070479DF87900BA
:104EE800F7E79DF87A00F4E79DF87B00F1E79DF875
:104EF8007C00EEE79DF87D00EBE79DF87E00E8E793
:104F08009DF87F00E5E79DF88000E2E79DF88100C5
:104F1800DFE79DF88200DCE79DF88300D9E79DF87C
:104F28008400D6E79DF88500D3E79DF88600D0E792
:104F38009DF88700CDE79DF88800CAE79DF88900AD
:104F4800C7E79DF88A00C4E79DF88B00C1E79DF884
:104F58008C00BEE79DF88D00BBE79DF88E00B8E792
:104F68009DF88F00B5E79DF89000B2E79DF8910095
:104F7800AFE79DF89200ACE79DF89300A9E79DF88C
:104F88009400A6E79DF89500A3E79DF89600A0E792
:104F98009DF897009DE79DF898009AE79DF899007D
:104FA80097E79DF89A0094E79DF89B0091E79DF894
:104FB8009C008EE79DF89D008BE79DF89E0088E792
:104FC8009DF89F0085E79DF8A00082E79DF8A10065
:104FD8007FE79DF8A2007CE79DF8A30079E79DF89C
:104FE800A40076E79DF8A50073E79DF8A60070E792
:104FF8009DF8A7006DE79DF8A8006AE79DF8A9004D
:1050080067E79DF8AA0064E79DF8AB0061E79DF8A3
:10501800AC005EE79DF8AD005BE79DF8AE0058E791
:105028009DF8AF0055E79DF8B00052E79DF8B10034
:105038004FE79DF8B2004CE79DF8B30049E79DF8AB
:10504800B40046E79DF8B50043E79DF8B60040E791
:105058009DF8B7003DE7024804F012FA002038E74F
:105068006CB8000884B008B50DF1080E8EE80F0082
:105078009DF848303F2B00F2E580DFE803F0E0DDE3
:10508800DAD7D4D1CECBC8C5C2BFBCB9B6B3B0ADE0
:10509800AAA7A4A19E9B9895928F8C898683807DD0
:1050A8007A7774716E6B6865625F5C595653504DC0
:1050B8004A4744413E3B3835322F2C2926209DF85B
:1050C8000800BDE8084004B070479DF80900F8E7FB
:1050D8009DF80A00F5E79DF80B00F2E79DF80C0033
:1050E800EFE79DF80D00ECE79DF80E00E9E79DF865
:1050F8000F00E6E79DF81000E3E79DF81100E0E7F0
:105108009DF81200DDE79DF81300DAE79DF814001A
:10511800D7E79DF81500D4E79DF81600D1E79DF86C
:105128001700CEE79DF81800CBE79DF81900C8E7EF
:105138009DF81A00C5E79DF81B00C2E79DF81C0002
:10514800BFE79DF81D00BCE79DF81E00B9E79DF874
:105158001F00B6E79DF82000B3E79DF82100B0E7EF
:105168009DF82200ADE79DF82300AAE79DF82400EA
:10517800A7E79DF82500A4E79DF82600A1E79DF87C
:1051880027009EE79DF828009BE79DF8290098E7EF
:105198009DF82A0095E79DF82B0092E79DF82C00D2
:1051A8008FE79DF82D008CE79DF82E0089E79DF884
:1051B8002F0086E79DF8300083E79DF8310080E7EF
:1051C8009DF832007DE79DF833007AE79DF83400BA
:1051D80077E79DF8350074E79DF8360071E79DF88C
:1051E80037006EE79DF838006BE79DF8390068E7EF
:1051F8009DF83A0065E79DF83B0062E79DF83C00A2
:105208005FE79DF83D005CE79DF83E0059E79DF893
:105218003F0056E79DF8400053E79DF8410050E7EE
:105228009DF842004DE79DF843004AE79DF8440089
:1052380047E79DF8450044E79DF8460041E79DF89B
:1052480047003EE7024804F01BF9002039E700BF99
:105258006CB8000884B008B50DF1080E8EE80F0090
:105268009DF848301F2B74D8DFE803F01016191C7E
:105278001F2225282B2E3134373A3D404346494CCE
:105288004F5255585B5E6164676A6D709DF80900FE
:10529800BDE8084004B070479DF80B00F8E79DF89A
:1052A8000D00F5E79DF80F00F2E79DF81100EFE714
:1052B8009DF81300ECE79DF81500E9E79DF8170045
:1052C800E6E79DF81900E3E79DF81B00E0E79DF885
:1052D8001D00DDE79DF81F00DAE79DF82100D7E7FC
:1052E8009DF82300D4E79DF82500D1E79DF8270015
:1052F800CEE79DF82900CBE79DF82B00C8E79DF87D
:105308002D00C5E79DF82F00C2E79DF83100BFE7E3
:105318009DF83300BCE79DF83500B9E79DF83700E4
:10532800B6E79DF83900B3E79DF83B00B0E79DF874
:105338003D00ADE79DF83F00AAE79DF84100A7E7CB
:105348009DF84300A4E79DF84500A1E79DF84700B4
:105358009EE7024804F094F8002099E76CB800082A
:1053680010B5204C00212078FFF7B6FA60780121AB
:10537800FFF7B2FAA0780221FFF7AEFAE07803212E
:10538800FFF7AAFA20790421FFF7A6FA607900212D
:10539800FFF708FC0121A079FFF704FCE079FFF78B
:1053A80059FB207A0021FFF7F3FA607A0121FFF711
:1053B800EFFAA07A0221FFF7EBFAE07A0321FFF770
:1053C800E7FA207B0421FFF7E3FA607B0021FFF76F
:1053D8003DFCA07B0121FFF739FCE07BBDE81040D4
:1053E800FFF78EBBC40C0020F0B543788FB004469D
:1053F8006C2B00F2C482DFE813F06D009200A80065
:10540800C000D800F00008012001380149016101FD
:1054180079019101A901C101C202D901DD01E101AE
:10542800E501E901EE01F301F801FD0102020702BD
:10543800C202C202C2020C02110216021B022002A0
:1054480027022C02310236023B02400245024A0280
:105458004F02540259025E02630268026D02720230
:1054680077027C02810286028B02900295029A02E0
:105478009F02A402C202C202C202A902C402DA0244
:10548800F00206031C03320348035E0374038A0315
:10549800C202C202C202A003B603CC03E203F803AD
:1054A8000E0424045F0475048B04A104B704CD041E
:1054B800E304F9040F0525053B05510567057D053E
:1054C8009305A905BF05D5050F0625063B06510618
:1054D80067067D06BE23037000234370D94BC21CA8
:1054E80003F1280153F8040B8B4242F8040BF9D15D
:1054F8001B88601C1380A178CD1C0231C9B203F04F
:1055080002F8EB2260552046A37823441A71A1784B
:105518000531C9B20FB0BDE8F040FFF76DBC14F813
:10552800030F0021FFF7D8F90123224640F6B821DE
:10553800A02002F0F7F9042322464FF42861A020A6
:105548000FB0BDE8F04002F0EDB90025861C01352A
:10555800EDB2294616F8010FFFF7BEF9042DF6D172
:1055680003342B46224640F6B921A02002F0DAF98E
:105578002B46224640F68421E1E70025861C0135AA
:10558800EDB2294616F8010FFFF7A6F9042DF6D15A
:1055980003342B46224640F6B921A02002F0C2F976
:1055A8002B46224640F68821C9E70021C078FFF73C
:1055B800F9FA20790121FFF7F5FA0334A078FFF70B
:1055C80049FA0323224640F6BD21A02002F0AAF999
:1055D8000423224640F68C21B1E70021C078FFF76A
:1055E800E1FA20790121FFF7DDFA0334A078FFF70B
:1055F80031FA0323224640F6BD21A02002F092F999
:10560800042322464FF4296199E70021C078FFF767
:10561800C9FA20790121FFF7C5FA0334A078FFF70A
:1056280019FA0323224640F6BD21A02002F07AF998
:105638000423224640F6942181E70021C078FFF731
:10564800B1FA20790121FFF7ADFA0334A078FFF70A
:1056580001FA0323224640F6BD21A02002F062F998
:105668000423224640F6982169E714F8030F002125
:10567800FFF78EF9012322464FF42C61A02002F097
:1056880051F90423224640F69C2158E70025861C40
:105698000135EDB2294616F8010FFFF779F9042D07
:1056A800F6D103342B46224640F6C121A02002F051
:1056B80039F92B4622464FF42A6140E70025861C1B
:1056C8000135EDB2294616F8010FFFF761F9042DEF
:1056D800F6D103342B46224640F6C121A02002F021
:1056E80021F92B46224640F6A42128E70021C0785C
:1056F800FFF7ACFA20790121FFF7A8FA0334A07864
:10570800FFF7FEF90323224640F6C521A02002F048
:1057180009F90423224640F6A82110E70021C078A1
:10572800FFF794FA20790121FFF790FA0334A07863
:10573800FFF7E6F90323224640F6C521A02002F030
:10574800F1F80423224640F6AC21F8E60021C0789F
:10575800FFF77CFA20790121FFF778FA0334A07863
:10576800FFF7CEF90323224640F6C521A02002F018
:10577800D9F8042322464FF42B61E0E60021C078D3
:10578800FFF764FA20790121FFF760FA0334A07863
:10579800FFF7B6F90323224640F6C521A02002F000
:1057A800C1F80423224640F6B421C8E64023C21CAF
:1057B8000021C4E64023C21C1946C0E64023C21C8F
:1057C8008021BCE64023C21CC021B8E64023C21C8D
:1057D8004FF48071B3E64023C21C4FF4A071AEE6CB
:1057E8004023C21C4FF4C071A9E64023C21C4FF4E9
:1057F800E071A4E64023C21C4FF400719FE64023E9
:10580800C21C4FF410719AE64023C21C4FF4207159
:1058180095E64023C21C4FF4307190E64023C21C29
:105828004FF440718BE64023C21C4FF4507186E65A
:105838004023C21C4FF4607181E64023C21C4FF420
:1058480070717CE61A0900204023C21C4FF4806165
:1058580075E64023C21C4FF4886170E64023C21CE1
:105868004FF490616BE64023C21C4FF4986166E6E2
:105878004023C21C4FF4A06161E64023C21C4FF4D0
:10588800A8615CE64023C21C4FF4B06157E6402390
:10589800C21C4FF4B86152E64023C21C4FF4C061E9
:1058A8004DE64023C21C4FF4C86148E64023C21CA1
:1058B8004FF4D06143E64023C21C4FF4D8613EE662
:1058C8004023C21C4FF4E06139E64023C21C4FF468
:1058D800E86134E64023C21C4FF4F0612FE6402310
:1058E800C21C4FF4F8612AE64023C21C4FF4006141
:1058F80025E64023C21C4FF4046120E64023C21C65
:105908004FF408611BE64023C21C4FF40C6116E6F5
:105918004023C21C4FF4106111E64023C21C4FF40F
:1059280014610CE64023C21C4FF4186107E64023BB
:10593800C21C4FF41C6102E64023C21C4FF42061D4
:10594800FDE54023C21C4FF42461F8E56F46C849C1
:105958000C90D1F800C0D1F804E08A68CB6801F156
:10596800100501F140043E4628686968083503C6F9
:10597800A5423746F7D160467146FFF745FA0FB0A2
:10598800F0BD6F46BB490C90D1F800C0D1F804E0D7
:105998008A68CB6801F1100501F140043E46286889
:1059A8006968083503C6A5423746F7D1E3E76F466D
:1059B800B1490C90D1F800C0D1F804E08A68CB68EE
:1059C80001F1100501F140043E4628686968083570
:1059D80003C6A5423746F7D1CDE76F46A7490C90D5
:1059E800D1F800C0D1F804E08A68CB6801F110054D
:1059F80001F140043E4628686968083503C6A54297
:105A08003746F7D1B7E76F469D490C90D1F800C0EB
:105A1800D1F804E08A68CB6801F1100501F140046F
:105A28003E4628686968083503C6A5423746F7D157
:105A3800A1E76F4693490C90D1F800C0D1F804E073
:105A48008A68CB6801F1100501F140043E462868D8
:105A58006968083503C6A5423746F7D18BE76F4614
:105A680089490C90D1F800C0D1F804E08A68CB6865
:105A780001F1100501F140043E46286869680835BF
:105A880003C6A5423746F7D175E76F467F490C90A4
:105A9800D1F800C0D1F804E08A68CB6801F110059C
:105AA80001F140043E4628686968083503C6A542E6
:105AB8003746F7D15FE76F4675490C90D1F800C0BB
:105AC800D1F804E08A68CB6801F1100501F14004BF
:105AD8003E4628686968083503C6A5423746F7D1A7
:105AE80049E76F466B490C90D1F800C0D1F804E043
:105AF8008A68CB6801F1100501F140043E46286828
:105B08006968083503C6A5423746F7D133E76F46BB
:105B180061490C90D1F800C0D1F804E08A68CB68DC
:105B280001F1100501F140043E462868696808350E
:105B380003C6A5423746F7D11DE76F4657490C9073
:105B4800D1F800C0D1F804E08A68CB6801F11005EB
:105B580001F140043E4628686968083503C6A54235
:105B68003746F7D107E76F464D490C90D1F800C08A
:105B7800D1F804E08A68CB6801F1100501F140040E
:105B88003E4628686968083503C6A5423746F7D1F6
:105B9800F1E66F4643490C90D1F800C0D1F804E013
:105BA8008A68CB6801F1100501F140043E46286877
:105BB8006968083503C6A5423746F7D1DBE66F4664
:105BC80039490C90D1F800C0D1F804E08A68CB6854
:105BD80001F1100501F140043E462868696808355E
:105BE80003C6A5423746F7D1C5E66F462F490C9044
:105BF800D1F800C0D1F804E08A68CB6801F110053B
:105C080001F140043E4628686968083503C6A54284
:105C18003746F7D1AFE66F4625490C90D1F800C05A
:105C2800D1F804E08A68CB6801F1100501F140045D
:105C38003E4628686968083503C6A5423746F7D145
:105C480099E66F461B490C90D1F800C0D1F804E0E2
:105C58008A68CB6801F1100501F140043E462868C6
:105C68006968083503C6A5423746F7D183E600BF01
:105C78004409002054040020840C0020140500204E
:105C880054030020840B0020140D00205408002029
:105C9800D408002094070020440C00209408002019
:105CA800840A0020D405002014070020D40C00200A
:105CB80054060020D40200206F46C5490C90D1F844
:105CC80000C0D1F804E08A68CB6801F1100501F141
:105CD80040043E4628686968083503C6A542374629
:105CE800F7D148E66F46BB490C90D1F800C0D1F80F
:105CF80004E08A68CB6801F1100501F140043E46D2
:105D080028686968083503C6A5423746F7D132E6E0
:105D18006F46B1490C90D1F800C0D1F804E08A6808
:105D2800CB6801F1100501F140043E462868696816
:105D3800083503C6A5423746F7D11CE66F46A74982
:105D48000C90D1F800C0D1F804E08A68CB6801F162
:105D5800100501F140043E4628686968083503C605
:105D6800A5423746F7D106E66F469D490C90D1F813
:105D780000C0D1F804E08A68CB6801F1100501F190
:105D880040043E4628686968083503C6A542374678
:105D9800F7D1F0E56F4693490C90D1F800C0D1F8DF
:105DA80004E08A68CB6801F1100501F140043E4621
:105DB80028686968083503C6A5423746F7D1DAE589
:105DC8006F4689490C90D1F800C0D1F804E08A6880
:105DD800CB6801F1100501F140043E462868696866
:105DE800083503C6A5423746F7D1C4E56F467F4953
:105DF8000C90D1F800C0D1F804E08A68CB6801F1B2
:105E0800100501F140043E4628686968083503C654
:105E1800A5423746F7D1AEE56F4675490C90D1F8E3
:105E280000C0D1F804E08A68CB6801F1100501F1DF
:105E380040043E4628686968083503C6A5423746C7
:105E4800F7D198E56F466B490C90D1F800C0D1F8AE
:105E580004E08A68CB6801F1100501F140043E4670
:105E680028686968083503C6A5423746F7D182E530
:105E78006F4661490C90D1F800C0D1F804E08A68F7
:105E8800CB6801F1100501F140043E4628686968B5
:105E9800083503C6A5423746F7D16CE56F46574922
:105EA8000C90D1F800C0D1F804E08A68CB6801F101
:105EB800100501F140043E4628686968083503C6A4
:105EC800A5423746F7D156E56F464D490C90D1F8B3
:105ED80000C0D1F804E08A68CB6801F1100501F12F
:105EE80040043E4628686968083503C6A542374617
:105EF800F7D140E56F4643490C90D1F800C0D1F87E
:105F080004E08A68CB6801F1100501F140043E46BF
:105F180028686968083503C6A5423746F7D12AE5D7
:105F28006F4639490C90D1F800C0D1F804E08A686E
:105F3800CB6801F1100501F140043E462868696804
:105F4800083503C6A5423746F7D114E56F462F49F1
:105F58000C90D1F800C0D1F804E08A68CB6801F150
:105F6800100501F140043E4628686968083503C6F3
:105F7800A5423746F7D1FEE46F4625490C90D1F883
:105F880000C0D1F804E08A68CB6801F1100501F17E
:105F980040043E4628686968083503C6A542374666
:105FA800F7D1E8E46F461B490C90D1F800C0D1F84E
:105FB80004E08A68CB6801F1100501F140043E460F
:105FC80028686968083503C6A5423746F7D1D2E480
:105FD800040A0020C409002094030020040B0020B8
:105FE8001406002054050020840900209402002093
:105FF800C40B002054070020D4030020D404002040
:106008001403002094040020440B00209405002071
:10601800D4060020140400206F4641490C90D1F8A2
:1060280000C0D1F804E08A68CB6801F1100501F1DD
:1060380040043E4628686968083503C6A5423746C5
:10604800F7D198E46F4637490C90D1F800C0D1F8E1
:1060580004E08A68CB6801F1100501F140043E466E
:1060680028686968083503C6A5423746F7D182E42F
:106078006F462D490C90D1F800C0D1F804E08A6829
:10608800CB6801F1100501F140043E4628686968B3
:10609800083503C6A5423746F7D16CE46F46234955
:1060A8000C90D1F800C0D1F804E08A68CB6801F1FF
:1060B800100501F140043E4628686968083503C6A2
:1060C800A5423746F7D156E46F4619490C90D1F8E6
:1060D80000C0D1F804E08A68CB6801F1100501F12D
:1060E80040043E4628686968083503C6A542374615
:1060F800F7D140E46F460F490C90D1F800C0D1F8B1
:1061080004E08A68CB6801F1100501F140043E46BD
:1061180028686968083503C6A5423746F7D12AE4D6
:10612800D40700201408002094060020C40A002088
:10613800040C0020440A00202DE9F0410446A8B0D0
:106148004578642200210FA802F0BDFC237828AA14
:106158008DF83C30A3788DF83D508DF83E301A44C8
:1061680023441B7902F8603C6C2D01F2A383DFE81D
:1061780015F06D0079009B0009017201E9013C02EC
:106188008F02E202FB028703EF03420495040B052A
:10619800A10B5E0574058A05A005B605CC05E205C8
:1061A800F8050E0624063A06A10BA10BA10B500612
:1061B80066067C069206CF06E506FB06110727074A
:1061C8003D07530769077F079507AB07C107D7073F
:1061D800ED07030819082F0845085B089708AD085C
:1061E800C308D908EF0805091B093109A10BA10B40
:1061F800A10B4709540961096E097B0988099509AA
:10620800A209AF09BC09C909A10BA10BA10BD609A9
:10621800E309F009FD090A0A170A240A310A3E0AA5
:10622800830A900A9D0AAA0AB70AC40AD10ADE0A92
:10623800EB0AF80A050B120B1F0B2C0B390B460B3C
:10624800530B600B6D0B7A0B870B940BE278AE49FE
:106258000DF13F0002F02CFC0FA8FFF7C5F828B09D
:10626800BDE8F081EE46E278A84BA94D9A71E37833
:1062780005F110060C93D5F80080D5F804C0AA687B
:10628800EB684035774630687168083603C7AE4218
:10629800BE46F7D140466146FEF7DCFDE070A278C5
:1062A800214605320FA8D5E7EE46D4F80320974BD0
:1062B800984DC3F80720E37805F110060C93D5F83C
:1062C8000080D5F804C0AA68EB6840357746306886
:1062D8007168083603C7AE42BE46F7D140466146EC
:1062E800FEF7B8FDEE4623798B4DE0700C93D5F898
:1062F8000080D5F804C0AA68EB6805F1100640359F
:10630800774630687168083603C7AE42BE46F7D193
:1063180040466146FEF79EFDEE4663797F4D20714B
:106328000C93D5F80080D5F804C0AA68EB6805F18D
:1063380010064035774630687168083603C7AE42A4
:10634800BE46F7D140466146FEF784FDEE46A37986
:10635800734D60710C93D5F80080D5F804C0AA6815
:10636800EB6805F1100640357746306871680836E5
:1063780003C7AE42BE46F7D140466146FEF76AFD06
:10638800A0718CE7EE46D4F80320604B654DC3F846
:106398000B20E37805F110060C93D5F80080D5F8AA
:1063A80004C0AA68EB6840357746306871680836DB
:1063B80003C7AE42BE46F7D140466146FEF74AFDE6
:1063C800EE462379584DE0700C93D5F80080D5F847
:1063D80004C0AA68EB6805F11006403577463068B6
:1063E8007168083603C7AE42BE46F7D140466146DB
:1063F800FEF730FDEE4663794C4D20710C93D5F8CD
:106408000080D5F804C0AA68EB6805F1100640358D
:10641800774630687168083603C7AE42BE46F7D182
:1064280040466146FEF716FDEE46A379404D607181
:106438000C93D5F80080D5F804C0AA68EB6805F17C
:1064480010064035774630687168083603C7AE4293
:10645800BE46F7D190E72346EE4633F8031F354A88
:10646800354D11809B7805F110069370E37840351F
:106478000C9355F8408C55F83CCC55F8382C55F809
:10648800343C774630687168083603C7AE42BE466A
:10649800F7D140466146FEF7DDFEEE462379274DEB
:1064A800E0700C93D5F80080D5F804C0AA68EB68B2
:1064B80005F110064035774630687168083603C71D
:1064C800AE42BE46F7D140466146FEF7C3FEEE46F1
:1064D80063791B4D20710C93D5F80080D5F804C062
:1064E800AA68EB6805F11006403577463068716890
:1064F800083603C7AE42BE46F7D140466146FEF7AE
:10650800B1FD6071CBE600BF1A0900201409002014
:106518004409002054040020840C002014050020A5
:1065280054030020840B0020140D00205408002080
:10653800D40800202309002094070020440C0020E0
:10654800940800202346EE4633F8031FBA4ABB4D91
:1065580011809B7805F110069370E37840350C9311
:1065680055F8408C55F83CCC55F8382C55F8343C47
:10657800774630687168083603C7AE42BE46F7D121
:1065880040466146FEF766FEEE462379AC4DE07064
:106598000C93D5F80080D5F804C0AA68EB6805F11B
:1065A80010064035774630687168083603C7AE4232
:1065B800BE46F7D140466146FEF74CFEEE4663798B
:1065C800A04D20710C93D5F80080D5F804C0AA68B6
:1065D800EB6805F110064035774630687168083673
:1065E80003C7AE42BE46F7D187E72346EE4633F8E7
:1065F800031F954A954D11809B7805F110069370FD
:10660800E37840350C9355F8408C55F83CCC55F858
:10661800382C55F8343C774630687168083603C71B
:10662800AE42BE46F7D140466146FEF713FEEE463F
:106638002379874DE0700C93D5F80080D5F804C015
:10664800AA68EB6805F1100640357746306871682E
:10665800083603C7AE42BE46F7D140466146FEF74C
:10666800F9FDEE4663797B4D20710C93D5F80080D7
:10667800D5F804C0AA68EB6805F1100640357746DE
:1066880030687168083603C7AE42BE46F7D134E7B2
:106698002346EE4633F8031F6F4A704D11809B78EE
:1066A80005F110069370E37840350C9355F8408C4B
:1066B80055F83CCC55F8382C55F8343C77463068BA
:1066C8007168083603C7AE42BE46F7D140466146F8
:1066D800FEF7C0FDEE462379614DE0700C93D5F8C6
:1066E8000080D5F804C0AA68EB6805F110064035AB
:1066F800774630687168083603C7AE42BE46F7D1A0
:1067080040466146FEF7A6FDEE466379554D207179
:106718000C93D5F80080D5F804C0AA68EB6805F199
:1067280010064035774630687168083603C7AE42B0
:10673800BE46F7D1E1E6EE46E2784B4B4B4DDA76B2
:10674800E37805F110060C93D5F80080D5F804C05D
:10675800AA68EB684035774630687168083603C721
:10676800AE42BE46F7D195E5EE46D4F803203E4B3F
:106778003F4DDA61E37805F110060C93D5F80080F7
:10678800D5F804C0AA68EB68403577463068716868
:10679800083603C7AE42BE46F7D140466146FEF70B
:1067A80059FBEE462379334DE0700C93D5F8008001
:1067B800D5F804C0AA68EB6805F11006403577469D
:1067C80030687168083603C7AE42BE46F7D1404606
:1067D8006146FEF73FFBEE466379274D20710C9327
:1067E800D5F80080D5F804C0AA68EB6805F1100652
:1067F8004035774630687168083603C7AE42BE46F2
:10680800F7D140466146FEF725FBEE46A3791B4DBE
:1068180060710C93D5F80080D5F804C0AA68EB68BD
:1068280005F110064035774630687168083603C7A9
:10683800AE42BE46F7D19FE526090020840A002013
:10684800D40500201407002029090020D40C0020BA
:1068580054060020D40200202C090020040A00203D
:10686800C40900209403002014090020040B002010
:1068780014060020540500208409002094020020FA
:10688800EE46D4F80320AF4BAF4D1A62E37805F11A
:1068980010060C93D5F80080D5F804C0AA68EB68F8
:1068A8004035774630687168083603C7AE42BE4641
:1068B800F7D140466146FEF7CDFAEE462379A34D5F
:1068C800E0700C93D5F80080D5F804C0AA68EB688E
:1068D80005F110064035774630687168083603C7F9
:1068E800AE42BE46F7D140466146FEF7B3FAEE46E1
:1068F8006379974D20710C93D5F80080D5F804C0C2
:10690800AA68EB6805F1100640357746306871686B
:10691800083603C7AE42BE46F7D140466146FEF789
:1069280099FAEE46A3798B4D60710C93D5F80080E7
:10693800D5F804C0AA68EB6805F11006403577461B
:1069480030687168083603C7AE42BE46F7D113E512
:106958002346EE4633F8031F7F4A804D11809B780B
:1069680005F110069370E37840350C9355F8408C88
:1069780055F83CCC55F8382C55F8343C77463068F7
:106988007168083603C7AE42BE46F7D14046614635
:10699800FEF760FCEE462379714DE0700C93D5F854
:1069A8000080D5F804C0AA68EB6805F110064035E8
:1069B800774630687168083603C7AE42BE46F7D1DD
:1069C80040466146FEF746FCEE466379654D207108
:1069D8000C93D5F80080D5F804C0AA68EB6805F1D7
:1069E80010064035774630687168083603C7AE42EE
:1069F800BE46F7D181E52346EE4633F8031F5A4ACF
:106A08005A4D11809B7805F110069370E378403554
:106A18000C9355F8408C55F83CCC55F8382C55F863
:106A2800343C774630687168083603C7AE42BE46C4
:106A3800F7D140466146FEF70DFCEE4623794C4DF2
:106A4800E0700C93D5F80080D5F804C0AA68EB680C
:106A580005F110064035774630687168083603C777
:106A6800AE42BE46F7D140466146FEF7F3FBEE461E
:106A78006379404D20710C93D5F80080D5F804C097
:106A8800AA68EB6805F110064035774630687168EA
:106A9800083603C7AE42BE46F7D12EE52346EE467A
:106AA80033F8031F344A354D11809B7805F11006E1
:106AB8009370E37840350C9355F8408C55F83CCCEE
:106AC80055F8382C55F8343C7746306871680836E4
:106AD80003C7AE42BE46F7D140466146FEF7BAFB51
:106AE800EE462379264DE0700C93D5F80080D5F852
:106AF80004C0AA68EB6805F110064035774630688F
:106B08007168083603C7AE42BE46F7D140466146B3
:106B1800FEF7A0FBEE4663791A4D20710C93D5F869
:106B28000080D5F804C0AA68EB6805F11006403566
:106B3800774630687168083603C7AE42BE46F7D15B
:106B4800DBE400BF14090020C40B00205407002018
:106B5800D4030020D40400203809002014030020A6
:106B680094040020440B00203B09002094050020D9
:106B7800D4060020140400203E090020D407002079
:106B880014080020940600202346EE4633F8031F1D
:106B9800CC4ACD4D11809B7805F110069370E378AF
:106BA80040350C9355F8408C55F83CCC55F8382CAA
:106BB80055F8343C774630687168083603C7AE42EA
:106BC800BE46F7D140466146FEF744FBEE462379C0
:106BD800BE4DE0700C93D5F80080D5F804C0AA68C3
:106BE800EB6805F11006403577463068716808365D
:106BF80003C7AE42BE46F7D140466146FEF72AFBC0
:106C0800EE466379B24D20710C93D5F80080D5F823
:106C180004C0AA68EB6805F110064035774630686D
:106C28007168083603C7AE42BE46F7D165E4A94A83
:106C3800E31C433453F8041BA34242F8041BF9D164
:106C4800A44B0DF13F0203F1400153F8040B8B42B2
:106C580042F8040BF9D1FFF7FFBA9F4AE31C43340B
:106C680053F8041BA34242F8041BF9D19A4B0DF1C7
:106C78003F0203F1400153F8040B8B4242F8040B26
:106C8800F9D1FFF7E9BA954AE31C433453F8041BDA
:106C9800A34242F8041BF9D1904B0DF13F0203F1D6
:106CA800400153F8040B8B4242F8040BF9D1FFF76B
:106CB800D3BA8B4AE31C433453F8041BA34242F86B
:106CC800041BF9D1864B0DF13F0203F1400153F843
:106CD800040B8B4242F8040BF9D1FFF7BDBA814A85
:106CE800E31C433453F8041BA34242F8041BF9D1B4
:106CF8007C4B0DF13F0203F1400153F8040B8B422A
:106D080042F8040BF9D1FFF7A7BA774AE31C4334DA
:106D180053F8041BA34242F8041BF9D1724B0DF13E
:106D28003F0203F1400153F8040B8B4242F8040B75
:106D3800F9D1FFF791BA6D4AE31C433453F8041BA9
:106D4800A34242F8041BF9D1684B0DF13F0203F14D
:106D5800400153F8040B8B4242F8040BF9D1FFF7BA
:106D68007BBA634AE31C433453F8041BA34242F83A
:106D7800041BF9D15E4B0DF13F0203F1400153F8BA
:106D8800040B8B4242F8040BF9D1FFF765BA594A54
:106D9800E31C433453F8041BA34242F8041BF9D103
:106DA800544B0DF13F0203F1400153F8040B8B42A1
:106DB80042F8040BF9D1FFF74FBA4F4AE31C4334AA
:106DC80053F8041BA34242F8041BF9D14A4B0DF1B6
:106DD8003F0203F1400153F8040B8B4242F8040BC5
:106DE800F9D1FFF739BA454AE31C433453F8041B79
:106DF800A34242F8041BF9D1404B0DF13F0203F1C5
:106E0800400153F8040B8B4242F8040BF9D1FFF709
:106E180023BA3B4AE31C433453F8041BA34242F809
:106E2800041BF9D1364B0DF13F0203F1400153F831
:106E3800040B8B4242F8040BF9D1FFF70DBA314A23
:106E4800E31C433453F8041BA34242F8041BF9D152
:106E58002C4B0DF13F0203F1400153F8040B8B4218
:106E680042F8040BF9D1FFF7F7B9274AE31C43347A
:106E780053F8041BA34242F8041BF9D1224B0DF12D
:106E88003F0203F1400153F8040B8B4242F8040B14
:106E9800F9D1FFF7E1B91D4AE31C433453F8041B49
:106EA800A34242F8041BF9D1184B0DF13F0203F13C
:106EB800400153F8040B8B4242F8040BF9D1FFF759
:106EC800CBB900BF41090020C40A0020040C0020EF
:106ED800440A00204409002054040020840C0020A7
:106EE8001405002054030020840B0020140D0020FA
:106EF80054080020D408002094070020440C0020E7
:106F080094080020840A0020D405002014070020DB
:106F1800D04AE31C433453F8041BA34242F8041B31
:106F2800F9D1CC4B0DF13F0203F1400153F8040BAA
:106F38008B4242F8040BF9D1FFF78EB9C64AE31C1D
:106F4800433453F8041BA34242F8041BF9D1C24B43
:106F58000DF13F0203F1400153F8040B8B4242F854
:106F6800040BF9D1FFF778B9BC4AE31C433453F852
:106F7800041BA34242F8041BF9D1B84B0DF13F02A0
:106F880003F1400153F8040B8B4242F8040BF9D18A
:106F9800FFF762B9B24AE31C433453F8041BA34217
:106FA80042F8041BF9D1AE4B0DF13F0203F1400149
:106FB80053F8040B8B4242F8040BF9D1FFF74CB994
:106FC800A84AE31C433453F8041BA34242F8041BA9
:106FD800F9D1A44B0DF13F0203F1400153F8040B22
:106FE8008B4242F8040BF9D1FFF736B99E4AE31CED
:106FF800433453F8041BA34242F8041BF9D19A4BBB
:107008000DF13F0203F1400153F8040B8B4242F8A3
:10701800040BF9D1FFF720B9944AE31C433453F821
:10702800041BA34242F8041BF9D1904B0DF13F0217
:1070380003F1400153F8040B8B4242F8040BF9D1D9
:10704800FFF70AB98A4AE31C433453F8041BA342E6
:1070580042F8041BF9D1864B0DF13F0203F14001C0
:1070680053F8040B8B4242F8040BF9D1FFF7F4B83C
:10707800804AE31C433453F8041BA34242F8041B20
:10708800F9D17C4B0DF13F0203F1400153F8040B99
:107098008B4242F8040BF9D1FFF7DEB8764AE31CBD
:1070A800433453F8041BA34242F8041BF9D1724B32
:1070B8000DF13F0203F1400153F8040B8B4242F8F3
:1070C800040BF9D1FFF7C8B86C4AE31C433453F8F2
:1070D800041BA34242F8041BF9D1684B0DF13F028F
:1070E80003F1400153F8040B8B4242F8040BF9D129
:1070F800FFF7B2B8624AE31C433453F8041BA342B7
:1071080042F8041BF9D15E4B0DF13F0203F1400137
:1071180053F8040B8B4242F8040BF9D1FFF79CB8E3
:10712800584AE31C433453F8041BA34242F8041B97
:10713800F9D1544B0DF13F0203F1400153F8040B10
:107148008B4242F8040BF9D1FFF786B84E4AE31C8C
:10715800433453F8041BA34242F8041BF9D14A4BA9
:107168000DF13F0203F1400153F8040B8B4242F842
:10717800040BF9D1FFF770B8444AE31C433453F8C1
:10718800041BA34242F8041BF9D1404B0DF13F0206
:1071980003F1400153F8040B8B4242F8040BF9D178
:1071A800FFF75AB83A4AE31C433453F8041BA34286
:1071B80042F8041BF9D1364B0DF13F0203F14001AF
:1071C80053F8040B8B4242F8040BF9D1FFF744B88B
:1071D800304AE31C433453F8041BA34242F8041B0F
:1071E800F9D12C4B0DF13F0203F1400153F8040B88
:1071F8008B4242F8040BF9D1FFF72EB8264AE31C5C
:10720800433453F8041BA34242F8041BF9D1224B20
:107218000DF13F0203F1400153F8040B8B4242F891
:10722800040BF9D1FFF718B81C4AE31C433453F890
:10723800041BA34242F8041BF9D1184B0DF13F027D
:1072480003F1400153F8040B8B4242F8040BF9D1C7
:10725800FFF702B8D40C002054060020D402002006
:10726800040A0020C409002094030020040B002015
:1072780014060020540500208409002094020020F0
:10728800C40B002054070020D4030020D40400209D
:107298001403002094040020440B002094050020CF
:1072A800D94AE31C433453F8041BA34242F8041B95
:1072B800F9D1D54B0DF13F0203F1400153F8040B0E
:1072C8008B4242F8040BF9D1FEF7C6BFCF4AE31C44
:1072D800433453F8041BA34242F8041BF9D1CB4BA7
:1072E8000DF13F0203F1400153F8040B8B4242F8C1
:1072F800040BF9D1FEF7B0BFC54AE31C433453F879
:10730800041BA34242F8041BF9D1C14B0DF13F0203
:1073180003F1400153F8040B8B4242F8040BF9D1F6
:10732800FEF79ABFBB4AE31C433453F8041BA3423D
:1073380042F8041BF9D1B74B0DF13F0203F14001AC
:1073480053F8040B8B4242F8040BF9D1FEF784BFC3
:10735800B14AE31C433453F8041BA34242F8041B0C
:10736800F9D1AD4B0DF13F0203F1400153F8040B85
:107378008B4242F8040BF9D1FEF76EBFA74AE31C13
:10738800433453F8041BA34242F8041BF9D1A34B1E
:107398000DF13F0203F1400153F8040B8B4242F810
:1073A800040BF9D1FEF758BF9D4AE31C433453F848
:1073B800041BA34242F8041BF9D1994B0DF13F027B
:1073C80003F1400153F8040B8B4242F8040BF9D146
:1073D800FEF742BF934AE31C433453F8041BA3420D
:1073E80042F8041BF9D18F4B0DF13F0203F1400124
:1073F80053F8040B8B4242F8040BF9D1FEF72CBF6B
:10740800894B0DF13F0203F1400153F8040B8B4205
:1074180042F8040BF9D1FEF71FBF844B0DF13F0270
:1074280003F1400153F8040B8B4242F8040BF9D1E5
:10743800FEF712BF7E4B0DF13F0203F1400153F8F6
:10744800040B8B4242F8040BF9D1FEF705BF794BC8
:107458000DF13F0203F1400153F8040B8B4242F84F
:10746800040BF9D1FEF7F8BE734B0DF13F0203F19F
:10747800400153F8040B8B4242F8040BF9D1FEF794
:10748800EBBE6E4B0DF13F0203F1400153F8040BC4
:107498008B4242F8040BF9D1FEF7DEBE684B0DF1C2
:1074A8003F0203F1400153F8040B8B4242F8040BEE
:1074B800F9D1FEF7D1BE634B0DF13F0203F1400154
:1074C80053F8040B8B4242F8040BF9D1FEF7C4BE03
:1074D8005D4B0DF13F0203F1400153F8040B8B4261
:1074E80042F8040BF9D1FEF7B7BE584B0DF13F0235
:1074F80003F1400153F8040B8B4242F8040BF9D115
:10750800FEF7AABE524B0DF13F0203F1400153F8BA
:10751800040B8B4242F8040BF9D1FEF79DBE4D4B8C
:107528000DF13F0203F1400153F8040B8B4242F87E
:10753800040BF9D1FEF790BE474B0DF13F0203F162
:10754800400153F8040B8B4242F8040BF9D1FEF7C3
:1075580083BE424B0DF13F0203F1400153F8040B87
:107568008B4242F8040BF9D1FEF776BE3C4B0DF185
:107578003F0203F1400153F8040B8B4242F8040B1D
:10758800F9D1FEF769BE374B0DF13F0203F1400117
:1075980053F8040B8B4242F8040BF9D1FEF75CBE9A
:1075A800314B0DF13F0203F1400153F8040B8B42BC
:1075B80042F8040BF9D1FEF74FBE2C4B0DF13F02F8
:1075C80003F1400153F8040B8B4242F8040BF9D144
:1075D800FEF742BE264B0DF13F0203F1400153F87E
:1075E800040B8B4242F8040BF9D1FEF735BE214B50
:1075F8000DF13F0203F1400153F8040B8B4242F8AE
:10760800040BF9D1FEF728BED4060020140400208C
:10761800D40700201408002094060020C40A002083
:10762800040C0020440A00204409002054040020CF
:10763800840C00201405002054030020840B002033
:10764800140D002054080020D408002094070020BE
:10765800440C002094080020840A0020D40500204F
:1076680014070020D40C002054060020D402002067
:10767800040A0020C4090020924B0DF13F0203F1D7
:10768800400153F8040B8B4242F8040BF9D1FEF782
:10769800E3BD8D4B0DF13F0203F1400153F8040B9C
:1076A8008B4242F8040BF9D1FEF7D6BD874B0DF19A
:1076B8003F0203F1400153F8040B8B4242F8040BDC
:1076C800F9D1FEF7C9BD824B0DF13F0203F140012C
:1076D80053F8040B8B4242F8040BF9D1FEF7BCBDFA
:1076E8007C4B0DF13F0203F1400153F8040B8B4230
:1076F80042F8040BF9D1FEF7AFBD774B0DF13F020D
:1077080003F1400153F8040B8B4242F8040BF9D102
:10771800FEF7A2BD714B0DF13F0203F1400153F892
:10772800040B8B4242F8040BF9D1FEF795BD6C4B64
:107738000DF13F0203F1400153F8040B8B4242F86C
:10774800040BF9D1FEF788BD664B0DF13F0203F13A
:10775800400153F8040B8B4242F8040BF9D1FEF7B1
:107768007BBD614B0DF13F0203F1400153F8040B5F
:107778008B4242F8040BF9D1FEF76EBD5B4B0DF15D
:107788003F0203F1400153F8040B8B4242F8040B0B
:10779800F9D1FEF761BD564B0DF13F0203F14001EF
:1077A80053F8040B8B4242F8040BF9D1FEF754BD91
:1077B800504B0DF13F0203F1400153F8040B8B428B
:1077C80042F8040BF9D1FEF747BD4B4B0DF13F02D0
:1077D80003F1400153F8040B8B4242F8040BF9D132
:1077E800FEF73ABD454B0DF13F0203F1400153F856
:1077F800040B8B4242F8040BF9D1FEF72DBD404B28
:107808000DF13F0203F1400153F8040B8B4242F89B
:10781800040BF9D1FEF720BD3A4B0DF13F0203F1FD
:10782800400153F8040B8B4242F8040BF9D1FEF7E0
:1078380013BD354B0DF13F0203F1400153F8040B22
:107848008B4242F8040BF9D1FEF706BD2F4B0DF120
:107858003F0203F1400153F8040B8B4242F8040B3A
:10786800F9D1FEF7F9BC2A4B0DF13F0203F14001B3
:1078780053F8040B8B4242F8040BF9D1FEF7ECBC29
:10788800244B0DF13F0203F1400153F8040B8B42E6
:1078980042F8040BF9D1FEF7DFBC1F4B0DF13F0294
:1078A80003F1400153F8040B8B4242F8040BF9D161
:1078B800FEF7D2BC4FF4D0621849194801F06CFDAC
:1078C800FEF7CABC94030020040B00201406002015
:1078D800540500208409002094020020C40B0020D5
:1078E80054070020D4030020D404002014030020EF
:1078F80094040020440B002094050020D4060020A6
:1079080014040020D4070020140800209406002046
:10791800C40A0020040C0020440A0020A3B8000870
:107928007CB800081FB50A248DE81C000A461023FD
:1079380001460548FAF7E6F904460520F9F754FC2C
:10794800204604B010BD00BF540D00201FB50A2406
:107958008DE81C000A46102301460548FAF762FA2A
:1079680004460520F9F740FC204604B010BD00BFCE
:10797800540D002010B54023DF4A0021A020FFF756
:10798800E5FF4023DD4A1946A020FFF7DFFF40232B
:10799800DB4A8021A020FFF7D9FF4023D94AC02124
:1079A800A020FFF7D3FF4023D74A4FF48071A020CF
:1079B800FFF7CCFF4023D54A4FF4A071A020FFF772
:1079C800C5FF4023D24A4FF4C071A020FFF7BEFF85
:1079D8004023D04A4FF4E071A020FFF7B7FF4023BF
:1079E800CD4A4FF40071A020FFF7B0FF4023CB4AE7
:1079F8004FF41071A020FFF7A9FF4023C84A4FF4A5
:107A08002071A020FFF7A2FF4023C64A4FF430712F
:107A1800A020FFF79BFF4023C34A4FF44071A020EA
:107A2800FFF794FF4023C14A4FF45071A020FFF79D
:107A38008DFF4023BE4A4FF46071A020FFF786FFF8
:107A48004023BC4A4FF47071A020FFF77FFF40230A
:107A5800B94A4FF48061A020FFF778FF4023B74A66
:107A68004FF48861A020FFF771FF4023B44A4FF418
:107A78009061A020FFF76AFF4023B24A4FF4986153
:107A8800A020FFF763FF4023AF4A4FF4A061A02076
:107A9800FFF75CFF4023AD4A4FF4A861A020FFF731
:107AA80055FF4023AA4A4FF4B061A020FFF74EFFCC
:107AB8004023A84A4FF4B861A020FFF747FF4023AE
:107AC800A54A4FF4C061A020FFF740FF4023A34A16
:107AD8004FF4C861A020FFF739FF4023A04A4FF4B4
:107AE800D061A020FFF732FF40239E4A4FF4D861AF
:107AF800A020FFF72BFF40239B4A4FF4E061A02012
:107B0800FFF724FF4023994A4FF4E861A020FFF7CC
:107B18001DFF4023964A4FF4F061A020FFF716FF9F
:107B28004023944A4FF4F861A020FFF70FFF402349
:107B3800914A4FF40061A020FFF708FF40238F4AC5
:107B48004FF40461A020FFF701FF40238C4A4FF453
:107B58000861A020FFF7FAFE40238A4A4FF40C611F
:107B6800A020FFF7F3FE4023874A4FF41061A020BE
:107B7800FFF7ECFE4023854A4FF41461A020FFF77D
:107B8800E5FE4023824A4FF41861A020FFF7DEFE8D
:107B98004023804A4FF41C61A0207F4CFFF7D6FE9B
:107BA80040237E4A4FF42061A020FFF7CFFE4023F8
:107BB8007B4A4FF42461A020FFF7C8FE2246012328
:107BC8004FF42861A020FFF7C1FE621C042340F691
:107BD8008421A020FFF7BAFE621D042340F6882105
:107BE800A020FFF7B3FE04F10902032340F68C211D
:107BF800A020FFF7ABFE04F10C0203234FF4296128
:107C0800A020FFF7A3FE04F10F02032340F69421FE
:107C1800A020FFF79BFE04F11202032340F69821EF
:107C2800A020FFF793FE04F11502012340F69C21E2
:107C3800A020FFF78BFE04F1160204234FF42A61FB
:107C4800A020FFF783FE04F11A02042340F6A421C2
:107C5800A020FFF77BFE04F11E02032340F6A821B3
:107C6800A020FFF773FE04F12102032340F6AC21A4
:107C7800A020FFF76BFE04F1240203234FF42B61CD
:107C8800A020FFF763FE04F12702464C032340F6C9
:107C9800B421A020FFF75AFE2246012340F6B8215E
:107CA800A020FFF753FE621C042340F6B921A02050
:107CB800FFF74CFE621D032340F6BD21A020FFF70D
:107CC80045FE04F1080201234FF42C61A020FFF7C0
:107CD8003DFE04F10902042340F6C121A020FFF76C
:107CE80035FE04F10D020323BDE8104040F6C5211E
:107CF800A020FFF72BBE00BF440900205404002039
:107D0800840C00201405002054030020840B00205C
:107D1800140D002054080020D408002094070020E7
:107D2800440C002094080020840A0020D405002078
:107D380014070020D40C002054060020D402002090
:107D4800040A0020C409002094030020040B00202A
:107D58001406002054050020840900209402002005
:107D6800C40B002054070020D4030020D4040020B2
:107D78001403002094040020440B002094050020E4
:107D8800D406002014040020D40700201408002082
:107D980094060020C40A00201A090020040C0020C0
:107DA800440A0020C40C002010B514460A230248D7
:107DB800FAF706FE204610BD0C0E002008B5026832
:107DC8000B4B9A4212D10B4A1368013313600A4ACB
:107DD800136801331360094B1B783BB1FBF72EFC8A
:107DE800132881BF064A13680133136008BD00BF1A
:107DF800001000403C020020380200204002002011
:107E08003402002002680E4B9A4217D10D490E4ADF
:107E1800097813780D48EB29C15404BF01200C4997
:107E280003F10103DBB208BF08703F2B88BF0023B2
:107E38000449137007480122FAF758BE704700BF7B
:107E4800004800404C0E0020B10E0020B40F002066
:107E5800080E00200C0E0020B0F5807F10B51BD155
:107E68002F4C237873B9AF222E492F4801F094FA8A
:107E780001232E4A137023702C4BBDE8104018784C
:107E8800FBF7C8BEB4222749274801F085FA00232A
:107E9800274A2370136010BDB0F5805F10D1204CC5
:107EA80023784BB9BD221F49224801F075FA0222F6
:107EB8001E4B1A700123DEE7C2221A491E48E4E766
:107EC800B0F5005F0DD1164C237833B9CB22154994
:107ED8001A4801F061FA0322EAE7D022114918484A
:107EE800D3E7B0F5804F0DD10D4B1A782AB904218C
:107EF8000E4A117001221A70BEE700220C491A704E
:107F08000A6010BDB0F5004FB6D1054B1A780AB912
:107F18000521EDE700221A70054B1A6010BD00BF5D
:107F28004002002020B90008B8B8000881020020EB
:107F380034020020CCB80008E1B80008F8B80008FE
:107F48000BB90008014B1870704700BF080E0020DD
:107F580010B592B03022002106A800F0B4FD14221A
:107F6800002101A800F0AFFD0123099310230A9313
:107F78000D230E93C32302240F93042306A8119301
:107F880006940C941094FAF759F80F2301930023E0
:107F980003934FF4A05304934FF48053032101A893
:107FA80002940593FAF71AFA12B010BD2DE9F04FB2
:107FB8000024A9B00AAE642200210FA8B54D00F034
:107FC80082FDF9F7E5F8FFF7C3FF142200213046D8
:107FD80000F079FD02942B6B224643F010032B63CB
:107FE8002B6B47F63D7103F010030293029B039439
:107FF8002B6BA94843F004032B632B6B012703F079
:1080080004030393039B04942B6B4FF00E0943F076
:1080180020032B632B6BDFF8BC8203F0200304934F
:10802800049B05942B6B4FF4E13B43F080032B63D7
:108038002B6BDFF8A4A203F080030593059B06943D
:108048002B6B43F001032B632B6B03F001030693A7
:10805800069B07942B6B43F002032B632B6B03F0F7
:1080680002030793079B08942B6B43F008032B63C9
:108078002B6B03F008030893089B09942B6B43F0C0
:1080880040032B632B6B03F040030993099BF9F71B
:10809800ADFB22464DF630418048F9F7A7FB224652
:1080A8004EF607017E48F9F7A1FB22464FF40F610F
:1080B8007C48F9F79BFB224640F2E1217A48F9F720
:1080C80095FB22464FF6CF017848F9F78FFB2246F9
:1080D80047F6FC217648F9F789FB47F63D733146A8
:1080E8006D480A930C940D940B97F9F797FA4DF68F
:1080F8003043314669480A930C940D940B97F9F76D
:108108008DFA4EF60703314665480A930C940D9490
:108118000B97F9F783FA4FF4E073314660480A93F6
:108128000B940C94F9F77AFA31465C480B940C944A
:10813800CDF82890F9F772FA4FF40F633146594891
:108148000A930C940D940B97F9F768FA40F2E1231F
:10815800314655480A930C940D940B97F9F75EFA3B
:108168004FF47043314650480A93CDF82C800C9751
:10817800F9F754FA4FF4807331464C480A93CDF816
:108188002C800C97F9F74AFA4FF6CF033146474847
:108198000A930C940D940B97F9F740FA47F6FC23D1
:1081A8004FF00C08314642480A930C940D940B97F3
:1081B800F9F734FA00942B6B3E4843F480032B63A1
:1081C8002B6B03F480030093009B01942B6B43F407
:1081D80000132B632B6B846003F400130193019B42
:1081E800354BC46080E8080804618461C461C0F844
:1081F8001480FAF7B7FB41F26F73304A50468AE8A9
:108208000C0009230A94CAF80C307460CAF80840B4
:10821800CAF81840FAF7CEFA314650460A940B9439
:10822800FAF7E2FA26482749274B284D80E80A0042
:108238004FF480438460C460036144618461C46115
:108248000462F9F7BBFC224B284685E80808AC60B5
:10825800EC602C61AC61EC61C5F81480FAF782FB24
:10826800224621462520F8F7E5FF2520F9F716F8DC
:10827800224621463620F8F7DDFF3620F9F70EF8BA
:10828800224621462720F8F7D5FF2720F9F706F8D8
:10829800224623E000380240001002400008024055
:1082A800001402400000024000040240000C02409A
:1082B80000180240740F0020001001400010004018
:1082C800540D0020005C0040801A06000C0E0020AF
:1082D8000048004000003110F40F002021462820FB
:1082E800F8F7A8FF2820F8F7D9FF224621461720DB
:1082F800F8F7A0FF1720F8F7D1FF224621463A20C9
:10830800F8F798FF3A20F8F7C9FF22462146462099
:10831800F8F790FF4620F8F7C1FF2246214640466D
:10832800F8F788FF4046F8F7B9FF22462146484645
:10833800F8F780FF4846F8F7B1FF5046FAF71EF9FC
:108348003A465E492846FAF7D1FB5D4800F016FB2D
:108358005C4B21461B68986801F09AF8FFF70AFB06
:10836800FAF7E2FE2046FBF755FC574B0FAC03F13A
:108378004005224618685968083303C2AB421446C0
:10838800F7D1FCF7EDFF514DDFF870814C4B9B683E
:10839800002B35DC2B78012B36D14D4B1B68642B19
:1083A80032D9DFF83C914B4F99F8021009F10100DE
:1083B80009EB01030231DA78C9B200F0BFF84C4684
:1083C800002870D1DFF838B13B7800F1010AC0B25B
:1083D800984262D3404801F053F899F802203F4888
:1083E8001444E178053200F0D7FF402200213C48D0
:1083F80000F069FB002038702870FAF70DFDC5E71A
:10840800384800F0C1FAC1E7FAF70CFD0128C8D0D6
:10841800354C2368C82B08D9344800F0BDFF344BCD
:108428001878FBF7F7FB00232360324C2368B3F579
:10843800FA7FABD93046FCF75DFC96E80300FCF701
:108448008DFCBE238DF83C306D238DF83D3008231C
:1084580030688DF83E30B388CDF83F000A210DF121
:108468003D00ADF8433000F04EF89DF83E3028AAA4
:108478001344EB228DF8470003F8602C9DF83E105A
:108488000FA80531C9B2FCF7B7FC4FF400414046CC
:10849800F9F7B1F90023236078E7215C584600F02A
:1084A8007BFF504690E7012803D14846FDF744FE7C
:1084B8009BE7114800F0E4FF97E700BF4C0E00204F
:1084C800381000200C00002094070020080E00201F
:1084D8003C0200208202002076B900083DB900085D
:1084E800410200200C0E00203402002078B9000858
:1084F80081020020380200206AB900080008024002
:1085080037B90008704710B5FF230446221AD2B2C3
:10851800914201D8184610BD14F8012B5340082287
:1085280013F0800F02F1FF324FEA430318BF83F0C4
:10853800310312F0FF02DBB2F2D1E7E730B5FF23D7
:1085480005462C1AE4B2A14203D89B1A5842584156
:1085580030BD15F8014B6340082413F0800F04F177
:10856800FF344FEA430318BF83F0310314F0FF04CC
:10857800DBB2F2D1E5E70000002182B00B4B00919D
:108588005A6C42F480425A645A6C02F48042009257
:10859800009A01911A6C42F080521A641B6C03F025
:1085A80080530193019B02B0704700BF003802401E
:1085B8002DE9F043044689B01422002103A800F0F5
:1085C80082FA2268224B9A423FD10025214C00951D
:1085D800236B4FF0120943F004032363236B4FF01E
:1085E800010803F004030093009B0195236B032704
:1085F80043F001032363236B042603F00103019373
:10860800019B4FF4007303A913480393CDF810900E
:10861800CDF8148006970796F9F700F84FF48073A1
:1086280003A90E480393CDF81090CDF8148006974F
:108638000796F8F7F3FF0295236C43F400032364CD
:10864800236C03F400030293029B09B0BDE8F08396
:10865800005C004000380240000802400000024070
:108668000268094B82B09A420BD100230193074B51
:108678001A6C42F010021A641B6C03F01003019389
:10868800019B02B0704700BF001000400038024054
:10869800142270B505468AB00DEB0200002100F0E7
:1086A80012FA2B684F4A934258D100264E4B019636
:1086B8005A6C05A942F010025A645A6C4B4802F0F1
:1086C80010020192019A02961A6B494C42F001027B
:1086D8001A631B6B03F001030293029B4FF4C06300
:1086E8000593022306930123079303230893072383
:1086F8000993F8F793FF4FF000633E49204684E85A
:108708000A004FF48063A660E66023616661A66193
:10871800E66126626662F8F7FBFD08B1FFF7F2FE34
:108728006C63354BA563354C23604FF00063636081
:1087380040234FF48062A36000232261E3606361F9
:10874800A361E361236263622046F8F7E1FD08B1A3
:10875800FFF7D8FE2C63A5630AB070BD284A934280
:10876800FAD10026204B03961A6C264842F4802240
:108778001A641A6C05A902F480220392039A0496DB
:108788001A6B214C42F002021A631B6B03F00203BE
:108798000493049B4FF4406305930223069301233B
:1087A80007930323089307230993F8F737FF4FF03C
:1087B8000063164A204684E80C004FF48063A660E4
:1087C800E66023616661A661E66126626662F8F783
:1087D8009FFD08B1FFF796FE6C630D4BA5630D4C2A
:1087E800A2E700BF0010014000380240000002402C
:1087F800140F002040640240B8640240B40E002008
:108808000048004000040240A80D002028600240F3
:1088180058600240500E00207047FEE7FEE7FEE772
:10882800FEE7704770477047F8F7CCBC0148F8F787
:108838003BBE00BFA80D00200148F8F735BE00BFB9
:10884800500E00204FF48070F8F7DCBF0148FAF7AB
:108858003BBA00BF740F002013B50A4C23681A688E
:10886800920604D559682046C9B200F0B3F800232F
:10887800019323681A6801925B680193019B02B017
:1088880010BD00BF0C0E002008B54FF48050F8F75B
:10889800B9FF4FF40050F8F7B5FF4FF48040F8F7F0
:1088A800B1FFBDE808404FF40040F8F7ABBF000047
:1088B8000148F9F777BE00BFF40F00200148F8F728
:1088C800F3BD00BF140F00200148F8F7EDBD00BF4D
:1088D800B40E002070B50E4615460C46A31B9D42EB
:1088E80001DC284670BDAFF3008004F8010BF5E702
:1088F80008B50A4B0246196809B909491960694659
:10890800186802448A4206D900F0A8F80C230360CC
:108918004FF0FF3008BD1A6008BD00BF8402002078
:10892800541800204FF0FF3070474FF400530020D8
:108938004B607047012070470020704700210C4BA6
:108948001A6842F001021A6099601A6822F084726B
:1089580022F480321A60074A5A601A6822F4802288
:108968001A604FF00062D960034B9A60704700BFED
:10897800003802401030002400ED00E0002343607E
:10898800036083607047000010B50F4A1178C9B2C0
:108998004B1CDBB213700D4B5A6803F10C00145CCE
:1089A8000132B2F5806FA8BF00225A609A68084861
:1089B800013A44549A6012B90120FFF7C3FABDE89E
:1089C80010400120F8F710BC820200203810002067
:1089D8004102002038B50B4C0D46A368B3F5806FF3
:1089E80001DBFFF7D1FF23685A1CB2F5806F2344DF
:1089F8001D7308BF0023226008BF2360A3680133EA
:108A0800A36038BD38100020DFF834D0002103E01F
:108A18000C4B5B58435004310B480C4B42189A429C
:108A2800F6D30B4A02E0002342F8043B094B9A4272
:108A3800F9D3FFF783FF00F017F8FFF7B7FA70478D
:108A48000000022078BC000800000020DC010020A3
:108A5800DC01002054180020FEE70000014B1868D4
:108A6800704700BF0C00002070B500250C4E0D4C5F
:108A7800A41BA410A54209D102F050FE00250A4EFD
:108A88000A4CA41BA410A54205D170BD56F8253088
:108A980098470135EEE756F8253098470135F2E753
:108AA80070BC000870BC000870BC000874BC0008EA
:108AB80010B5431E0A44914200D110BD11F8014B74
:108AC80003F8014FF7E703460244934200D1704789
:108AD80003F8011BF9E7002B2DE9F0471E46BBBF41
:108AE80003F100431E4600232D2388B0149F1299DA
:108AF80027F02007462F1446109DDDF84CA00B7078
:108B080004D0452F00D10135022300E0032307AA32
:108B1800049206AA03928DE828042246334600F000
:108B2800E7FE472F804602D1119BDB0726D5462F4B
:108B380008EB050911D198F80030302B0AD1002232
:108B4800002320463146F7F763FF18B9C5F1010540
:108B5800CAF80050DAF80030994400220023204671
:108B68003146F7F755FF38B93022079B994505D9A3
:108B7800591C07911A70F8E7CDF81C904046079BDE
:108B8800159AA3EB0803136008B0BDE8F087034605
:108B9800F7B5002903F8022BB6BF2D222B22494234
:108BA8000929427021DD0DF1070217460A2691FBBB
:108BB800F6F506FB1511092D01F1300102F8011C2B
:108BC80002F1FF34294609DC3031023A04F8011C6D
:108BD800BA421C4604D3201A03B0F0BD2246E6E789
:108BE80012F8011B03F8011BF2E730221C4611445E
:108BF80004F8022B5970EEE72DE9F04F91B00C46BE
:108C08001A9F93461E46054601F0C2FD03681846A2
:108C18000993F7F7D5FA00230E933B680A900733B8
:108C280023F0070303F1080294F81880D4F800A091
:108C38003A60D3E90023C4E91223D4F84C90A76C16
:108C480029F000430B934FF0FF32A64B38460B999F
:108C5800F7F710FF002840F0F7814FF0FF32A14BE3
:108C680038460B99F7F7E8FE002840F0ED8100221E
:108C7800002338464946F7F7D5FE10B12D2384F86E
:108C88004330994B994FB8F1470F98BF1F460323BC
:108C98004FF0000923612AF00403236000965B4625
:108CA8000FAA2146284600F0DFF9013040F09A80EB
:108CB8004FF0FF3011B0BDE8F08F62680EA8531C6A
:108CC8000DF1340E4AF4806341D10622626000211E
:108CD8002360019363680DF13302059002920093BB
:108CE8003A464B460691CDF81080CDF80CE0284660
:108CF800FFF7F1FE08F0DF03472B074609D10D9B6C
:108D0800D81C02DB6268934259DDA8F102085FFAB9
:108D180088F8B8F1650F0D9936D80139424604F143
:108D280050000D91FFF733FF0E9A81468318012AF0
:108D3800236102DC2268D10701D5013323619DF844
:108D48003330002BAAD02D2384F84330A6E7B8F19E
:108D5800670F02D0B8F1470FB9D19AB10021069137
:108D68000DF133018DE80C00236005903A46CDF8EB
:108D78001080CDF80CE002914B462846FFF7ABFE79
:108D88000746BCE70122A1E7B8F1660F19D100290F
:108D980063680CDD216113B92268D20702D501335B
:108DA8000B4423610D9B4FF00009A365C7E713B976
:108DB8002268D00701D50233F3E70123F1E74FF02A
:108DC80067080D9B0E9A934205DB22682361D10741
:108DD800E8D50133E5E7002BCCBF0123C3F102033B
:108DE8001344DEE723685A0507D423693A465946EF
:108DF8002846B04701302AD15AE7B8F1650F40F24A
:108E0800DC80D4E9120100220023F7F701FE0028D4
:108E180039D00123364A59462846B04701303FF435
:108E280047AF0E9B0D9A9A4202DB2368D8070ED5EE
:108E38000A9B099A59462846B04701303FF438AF93
:108E4800002704F11A080E9B013B9F4211DB23689F
:108E58009F0708D5002704F11908E3680F9A9B1AA1
:108E68009F42C0F2E780E0680F9B9842B8BF18465F
:108E780020E70123424659462846B04701303FF4CF
:108E880017AF0137DFE70D9B002B33DC0123184AAE
:108E980059462846B04701303FF40AAF0D9B23B925
:108EA8000E9B13B92368D907D1D50A9B099A59464D
:108EB8002846B04701303FF4FBAE4FF0000804F1FC
:108EC8001A090D9B5B42984501DB0E9B8EE7012337
:108ED8004A4659462846B04701303FF4E9AE08F102
:108EE8000108EEE7FFFFEF7FA8B90008ACB900085A
:108EF800B8B900080E9AA36D9A42A8BF1A46002A6C
:108F0800904636DC4FF0000A04F11A0328EAE878A4
:108F18000B93D4F85890A9EB08039A4531DB0E9BC4
:108F28000D9A9A4238DB2368DA0735D40E9B0D99DF
:108F3800A3EB0902A3EB01089045A8BF9046B8F13E
:108F4800000F31DC002728EAE87804F11A090D9AA5
:108F58000E9B9B1AA3EB08039F42BFF678AF012331
:108F68004A4659462846B04701303FF4A1AE01377A
:108F7800EDE7134659463A462846B0470130C1D175
:108F880096E601230B9A59462846B04701303FF42C
:108F98008FAE0AF1010ABCE70A9B099A594628468E
:108FA800B0470130C2D183E6434607EB0902594670
:108FB8002846B0470130C5D17AE60E9A012A01DC6D
:108FC800DB0734D501233A4659462846B0470130D5
:108FD8003FF46EAE0A9B099A59462846B0470130BD
:108FE8003FF466AED4E9120100220023F7F710FD22
:108FF80050B1002704F11A080E9B013B9F420CDB7D
:109008004B4604F15002F2E60E9B7A1C013B59468E
:109018002846B0470130F3D14AE601234246594673
:109028002846B04701303FF443AE0137E4E7012357
:109038003A46ECE70123424659462846B0470130F4
:109048003FF436AE013708E73A464B4638464946BC
:10905800F7F710FD00283FF430AE014B014F12E640
:10906800B0B90008B4B900082DE9F04791461F4689
:109078008A680B6906469342B8BF1346C9F80030A0
:1090880091F843200C46DDF8208012B10133C9F86D
:1090980000302368990642BFD9F800300233C9F876
:1090A8000030256815F0060507D104F1190AE368B0
:1090B800D9F800209B1A9D422ADB94F84330226895
:1090C800003318BF012392062FD404F14302394616
:1090D8003046C047013022D02368E56803F0060314
:1090E800042B18BF0025D9F800204FF0000908BF4D
:1090F800AD1AA368226908BF25EAE5759342C4BF83
:109108009B1AED181A344D451BD10020BDE8F08795
:109118000123524639463046C047013003D14FF04B
:10912800FF30BDE8F0870135C1E73020E11881F84C
:1091380043005A1C94F845102244023382F8431025
:10914800C3E70123224639463046C0470130E6D0FE
:1091580009F10109D7E700002DE9F04317460A7E17
:1091680085B06E2A984606460C460C9B01F1430EC4
:1091780000F0BC801AD8632A2ED00AD8002A00F042
:10918800C880582A00F08A8004F1420584F84220F9
:109198002AE0642A01D0692AF6D121681A6811F0F8
:1091A800800F23D0111D1960136827E0732A00F07F
:1091B800B48008D86F2A2AD0702AE5D10A6842F00C
:1091C80020020A6003E0752A21D0782ADCD17822AF
:1091D8006F4984F8452064E01A6801F14205111DC1
:1091E8001960136884F842300123A3E011F0400F9E
:1091F80002F104011960D7D0B2F90030002B03DA6C
:109208002D225B4284F8432062490A2217E0206835
:10921800196810F0800F03D0081D18600B6806E06D
:1092280010F0400F01F104001860F7D00B886F2A86
:1092380014BF0A2208225749002084F843006568B1
:10924800002DA560C0F29C80206820F004002060FA
:10925800002B3FD1002D40F095807546082A0BD190
:109268002368DA0708D5236962689A42DEBF30238B
:1092780005F8013C05F1FF35AEEB05032361CDF898
:1092880000803B4603AA21463046FFF7EDFE013039
:1092980055D14FF0FF3005B0BDE8F08381F8452087
:1092A8003C492268186812F0800F00F104051D601F
:1092B80001D0036802E05506FBD50388D00744BFF8
:1092C80042F0200222601BB9226822F020022260AC
:1092D8001022B1E77546B3FBF2F002FB1033CB5C0A
:1092E80005F8013D03460028F5D1B7E708681A6874
:1092F80010F0800F496904D0101D186013681960B8
:1093080007E010F0400F02F1040018601368F6D06F
:109318001980002375462361B1E71A68111D196089
:10932800156800216268284601F0ACFA08B1401BB4
:10933800606063682361002384F843309FE72369F2
:109348002A4639463046C0470130A2D023689B07D9
:1093580007D5002504F11909E368039A9B1A9D4271
:1093680005DBE068039B9842B8BF184693E70123E2
:109378004A4639463046C04701308AD00135EBE7C6
:10938800002BA7D10B7804F1420584F8423065E739
:10939800CBB90008BAB900080FB40A4B13B51C685A
:1093A80024B1A36913B9204601F068F905AB049A02
:1093B800A1682046019301F075FF02B0BDE8104096
:1093C80004B070470C00002070B50E46054618B171
:1093D80083690BB901F052F9AB69AC6813B9284637
:1093E80001F04CF9234B9C4217D16C68A3891B07E9
:1093F8001DD52369DBB1013EA36816F8011F013BA7
:10940800A360E9B9002B2EDA22460A21284600F08B
:1094180021F9013011D00A2070BD174B9C4201D1AF
:10942800AC68E3E7154B9C4208BFEC68DEE72146D1
:10943800284600F061F90028DDD04FF0FF3070BDFC
:10944800002B04DAA269934206DB0A2904D02368B8
:109458005A1C22601970CFE72246284600F0FAF815
:109468000130C9D1E9E70A2023685A1C2260187024
:1094780070BD00BF0CBA00082CBA0008ECB900088F
:10948800024B01461868FFF79FBF00BF0C00002081
:1094980000294FF480630CBF0222002200F000B8BC
:1094A8002DE9F7431D46514B04461E680F4690466A
:1094B80026B1B36913B9304601F0E0F84C4B9C4231
:1094C80052D17468B8F1020F06D0B8F1010F00F25A
:1094D8008980002DC0F286802146304601F064F86C
:1094E800616B41B104F14403994202D0304601F066
:1094F800B7FC002363630023A3616360A3891B0691
:1095080003D52169304601F0ABFCA389B8F1020FFD
:1095180023F44A6323F00303A3815DD001AB6A46B9
:109528002146304601F042F9A3891843A0812DBB9A
:10953800009D284601F09EF9074600284ED1DDF827
:109548000090A9453CD14FF0FF30A38943F00203B6
:10955800A3810023A36004F147032360236101234F
:10956800636103B0BDE8F083224B9C4201D1B4682B
:10957800A8E7214B9C4208BFF468A3E7002FD8D086
:10958800B36913B9304601F079F8B8F1010F08BF93
:10959800A389276004BF43F00103A381A38927613E
:1095A80013F0080065611BD013F001004FF00003B1
:1095B8001FBF6D42A360A561184608BFA560D0E72C
:1095C800484601F057F907460028BCD0A3894D4604
:1095D80043F08003A381D3E70020B6E7A946F5E767
:1095E800A060BEE74FF0FF30BBE700BF0C000020D3
:1095F8000CBA00082CBA0008ECB900080EB44FF4F5
:10960800027100B59CB0ADF814106FF000410491E0
:1096180007914FF6FF711DAB02900690084853F86A
:10962800042BADF81610006802A9019301F01EFD85
:109638000022029B1A701CB05DF804EB03B070475F
:109648000C000020034611F8012B03F8012B002A17
:10965800F9D17047F8B50E461446054618B1836926
:109668000BB901F00BF8214B9C422AD16C68A36915
:10967800A360A3891A072ED5236963B323692068D9
:10968800F6B2C01A63693746984204DB2146284679
:1096980000F08AFF28BBA3680130013BA360236860
:1096A8005A1C22601E706369984204D0A389DB07A4
:1096B80019D50A2E17D12146284600F075FF90B11A
:1096C8000FE00B4B9C4201D1AC68D0E7094B9C42A0
:1096D80008BFEC68CBE72146284600F00DF80028C3
:1096E800CCD04FF0FF373846F8BD00BF0CBA0008A1
:1096F8002CBA0008ECB90008324B70B51D68064654
:109708000C4625B1AB6913B9284600F0B7FF2E4BBC
:109718009C420FD16C68B4F90C309AB215072CD45E
:10972800D00611D40922326043F04003A3814FF0E0
:10973800FF3070BD254B9C4201D1AC68EBE7244B50
:109748009C4208BFEC68E6E7510712D5616B41B14E
:1097580004F14403994202D0304601F081FB002312
:109768006363A38923F02403A3810023636023692F
:109778002360A38943F00803A38123694BB9A38914
:1097880003F42073B3F5007F03D02146304601F07F
:1097980031F8A28912F001030CD00023A360636999
:1097A8005B42A361236953B9B4F90C3013F080000C
:1097B800BAD170BD920758BF6369A360F2E7002071
:1097C800F7E700BF0C0000200CBA00082CBA00080C
:1097D800ECB900082DE9F74F03690C6980469C42F3
:1097E80000F38280013C01F1140700F1140657F8D8
:1097F800245056F824000135B0FBF5F54FEA840EE5
:1098080006EB0E0307EB0E0901938DB34FF0000A28
:109818003846B446D34650F8042B93B205FB03A34D
:10982800120C4FEA134A05FB02A29BB2ABEB0303EF
:10983800BCF800B04FEA124A5B441FFA82FBDCF81E
:1098480000208145CBEB124202EB23429BB243EA54
:1098580002434FEA224B4CF8043BDCD256F80E3058
:1098680033B9019B043B9E421A4631D3C8F81040D5
:10987800404601F01EFA002826DB30464FF0000E65
:10988800013557F8041BD0F800C08BB2AEEB0303C8
:109898001FFA8CF213440A0CC2EB1C4202EB23425F
:1098A8009BB243EA0243B9454FEA224E40F8043BD3
:1098B800E7D256F8242006EB84032AB9043B9E42DB
:1098C8001A460BD3C8F81040284603B0BDE8F08FFD
:1098D8001268043B002AC9D1013CC4E71268043B62
:1098E800002AEFD1013CEAE70020EEE70000000083
:1098F8002DE9F04F466A95B00446219DCDE9022333
:109908003EB9102000F0B6FF6062466086600660CF
:10991800C660636A196851B15A68012393404A6066
:109928008B60204600F0F0FF0022636A1A60039BF8
:10993800002BB7BF012300232B60039BAEBF2B6016
:1099480023F000430393DDF80C90AB4B33EA090393
:109958001BD142F20F73209A1360029B23B9C9F3FB
:109968001300002800F08385229B53B9A34B21E004
:10997800A34B06930833229A1360069815B0BDE8E6
:10998800F08F9E4B06930333F5E7DDE9026700226B
:10999800002330463946F7F73BF8804660B101238B
:1099A800209A1360229B002B00F05E85954B229A2B
:1099B8001360013B0693E0E712AB019313AB0093EE
:1099C80032463B46204601F0EDF9C9F30A55824676
:1099D800002D7DD03046C7F3130343F07F5141F487
:1099E8004011A5F2FF35CDF840800022864BF6F7EE
:1099F800F3FB7BA3D3E90023F6F7A2FD7AA3D3E90F
:109A08000023F6F7EBFB064628460F46F6F732FD2D
:109A180077A3D3E90023F6F793FD02460B463046B9
:109A28003946F6F7DBFB06460F46F7F739F800220A
:109A38008346002330463946F6F7F4FF58B15846B6
:109A4800F6F718FD02460B4630463946F6F7E0FFB2
:109A580008B90BF1FF3BBBF1160F58D8DDE902231B
:109A68006A4901EBCB01D1E90001F6F7F9FF0028BB
:109A78004FD000230BF1FF3B0D93129B5D1B6B1E18
:109A8800079343BF0023C5F1010807934FF000086F
:109A9800BBF1000F3FDB079BCDF830B05B44079369
:109AA800002308931E9B092B00F2B480052BC4BF2A
:109AB800043B1E931E9BC8BF0026A3F10203D8BF18
:109AC8000126032B00F2B280DFE803F084862D78AC
:109AD800139B129D1D4405F23243202B11DD029A7F
:109AE80005F21240C3F1400322FA00F009FA03F329
:109AF8001843F6F7AFFC0123A1F1F871013D10936B
:109B080073E7C3F12000029B03FA00F0F1E7012399
:109B1800B2E70D90B1E7CBF1000308930023A8EB5F
:109B28000B080C93BEE7012309931F9B002B40F3FE
:109B380080809946049300220421656A6A6001F1D5
:109B480014029A427AD96968204600F0A9FE636A2D
:109B580028601B68B9F10E0F069300F2F080002E02
:109B680000F0ED80DDE90223BBF1000FCDE90E2303
:109B780079DD264A0BF00F034FEA2B1602EBC303DD
:109B8800F006D3E90023CDE90A235CD5DDE90E010F
:109B98001F4B0325D3E90823F6F7FCFDCDE90201A5
:109BA80006F00F061A4F002E4FD1DDE90A23DDE932
:109BB8000201F6F7EFFDCDE902016EE001230993FA
:109BC8001F9B5B4403F1010904934B46012BB8BF6B
:109BD8000123B0E70023A7E70023F0E7AFF30080F5
:109BE80061436F63A787D23FB3C8608B288AC63F9B
:109BF800FB799F501344D33F0000F07FE5B900087C
:109C0800DCB90008B9B900080000F83F78BA0008C4
:109C180050BA00080126002309961E934FF0FF331F
:109C280000220493994612231F9284E70123099383
:109C3800F4E70123049399461A46F5E76A68490050
:109C480001326A607BE70225ACE7F10708D5DDE958
:109C58000A01D7E90023F6F773FCCDE90A010135BB
:109C6800761008379FE700F0A580DDE90E01CBF1FB
:109C78000006A24B06F00F0203EBC203D3E9002350
:109C8800F6F75EFC02250023CDE902019C4F361150
:109C9800002E40F08480002B8DD10D9B002B00F00E
:109CA8008B80DDE90223CDE90A23DDE90A010022E0
:109CB800944BF6F7B7FE00287ED0B9F1000F7BD0A1
:109CC800049B002B37DDDDE90A0100228E4BF6F7F5
:109CD80037FCCDE90201049E0BF1FF370135284618
:109CE800F6F7C8FBDDE90223F6F72AFC874B0022CA
:109CF800F6F774FACDE90A010B9BA3F150750B95A1
:109D0800002E5CD1DDE902010022814BF6F764FAEE
:109D18000A9A2B46CDE90201F6F7A2FE002840F088
:109D2800F782DDE902010A9A05F10043F6F77AFEA7
:109D3800002840F0EB82DDE90E23CDE90223139BD6
:109D4800002BC0F25081BBF10E0F00F34C816B4B1E
:109D580003EBCB03D3E90023CDE904231F9B002B9E
:109D680080F2DA80B9F1000F00F3D68040F0CD829E
:109D7800DDE904010022664BF6F7E2FBDDE9022388
:109D8800F6F764FE4E464F46002840F0A482069B34
:109D9800069A5D1C31230BF1010B13709FE2F20749
:109DA80005D5D7E90023F6F7CBFB0123013576105B
:109DB80008376DE7022570E75F464E468FE7069A3B
:109DC8004E4B32441192099A711E002A48D003EB77
:109DD800C103D3E9002300204E49F6F7DBFCDDE997
:109DE8000A23F6F7F9F9CDE90A01069DDDE9020132
:109DF800F6F756FE0646F6F73DFB02460B46DDE94A
:109E08000201F6F7E9F9DDE90A23303605F8016BB6
:109E1800CDE90201F6F706FE002864D1DDE9022348
:109E280000203849F6F7D8F9DDE90A23F6F7FAFDF4
:109E3800002840F0B980119B9D423FF47CAFDDE9DA
:109E48000A010022304BF6F77BFB0022CDE90A011C
:109E5800DDE902012C4BF6F773FBCDE90201C5E7FA
:109E680003EBC101D1E90001DDE90A23F6F768FB3C
:109E7800CDE90A01069DDDE90201F6F711FE064665
:109E8800F6F7F8FA02460B46DDE90201F6F7A4F9FF
:109E98003036119B05F8016BAB42CDE902014FF05A
:109EA800000224D11B4BDDE90A01F6F797F90246B7
:109EB8000B46DDE90201F6F7D3FD002874D1DDE990
:109EC8000A2300201349F6F787F902460B46DDE915
:109ED8000201F6F7A7FD00283FF42DAF15F8013C65
:109EE8006A1E302B01D0BB464DE01546F6E7064BFF
:109EF800F6F726FBCDE90201BDE700BF78BA0008F6
:109F080050BA00080000F03F0000244000001C4048
:109F1800000014400000E03F069DDDE90267DDE92E
:109F2800042330463946F6F735FCF6F7B9FD804686
:109F3800F6F7A0FADDE90423F6F702FB02460B4622
:109F480030463946F6F748F908F1300605F8016B4E
:109F5800069E0246AE1BB1450B4637D1F6F73EF9D1
:109F680006460F4602460B46DDE90401F6F75AFDA0
:109F7800C8B9DDE9040132463B46F6F749FD10B1A0
:109F880018F0010F0FD15146204600F0BDFC002308
:109F9800209A2B700BF101031360229B002B3FF4D6
:109FA800ECAC1D60E9E45F4615F8012C6B1E392AFC
:109FB80006D1069A9A4207D1302313701346013707
:109FC8001A7801321A708EE71D46EDE70022B54B6C
:109FD800F6F7B6FA0022002306460F46F6F718FDF4
:109FE80000289CD0CFE7099A002A00F029811E9A00
:109FF800012A00F30E81109A002A00F0068103F26C
:10A0080033434546089E079A01211A44204698443E
:10A01800079200F019FD0746002D0BDD079B002B6A
:10A0280008DDAB42A8BF2B46079AA8EB0308ED1A38
:10A03800D31A0793089BFBB1099B002B00F00481FE
:10A04800002E11DD39463246204600F093FD524677
:10A0580001460746204600F000FD51460A9020467A
:10A0680000F052FC0A9B9A46089B9A1B04D0514662
:10A07800204600F07FFD82460121204600F0E4FCE6
:10A088000C9B0646002B40F3E1801A460146204609
:10A0980000F070FD1E9B0646012B40F3DA8000237A
:10A0A8000893336906EB8303186900F07FFCC0F15D
:10A0B8002000079B184410F01F0000F0F080C0F14A
:10A0C8002003042B40F3E280079BC0F11C0080446E
:10A0D800054403440793B8F1000F05DD5146424695
:10A0E800204600F095FD8246079B002B05DD314692
:10A0F8001A46204600F08CFD06460D9B002B00F00A
:10A10800D3803146504600F0D4FD002880F2CC8040
:10A11800002351460A22204600F00DFC099B0BF152
:10A12800FF3B8246002B00F0A981002339460A2212
:10A13800204600F000FC049B0746002B03DC1E9B16
:10A14800022B00F3B980002D05DD39462A4620464A
:10A1580000F05EFD0746089B002B00F0108179682F
:10A16800204600F09DFB05463A6907F10C010232D2
:10A1780092000C30FEF79CFC01222946204600F094
:10A1880047FD07970746029BDDF8188003F0010397
:10A19800089331465046FFF71DFB0799054600F125
:10A1A8003009504600F085FD3A4602903146204677
:10A1B80000F099FDC3680246002B40F0E28001469A
:10A1C8000990504600F075FD0346099A114620464D
:10A1D800099300F099FB099B002B40F0D4801E9A4C
:10A1E800002A40F0D080089A002A40F0CC80B9F1CB
:10A1F800390F00F0E880029B002B01DD05F13109E1
:10A2080008F1010588F800906BE0129BC3F1360352
:10A21800F7E6089B09F1FF36B342B7BF089B9E1BC0
:10A22800F21A0C9BBFBF08969B180C930026B9F135
:10A23800000FB9BFA8EB0905002345464B46E2E6E7
:10A24800089E4546099FE7E6089A10E71E9B012BE2
:10A2580018DC029BB3B9039BC3F31303A3B9039B95
:10A2680023F000431B0D1B052BB1079B08F10108C8
:10A2780001330793012308930C9B002B7FF411AF44
:10A28800012016E70023F6E7029BF4E73FF423AF2B
:10A29800079A1C331A4498441D4413461AE7034688
:10A2A800F6E700BF00002440B9F1000F33DC1E9B25
:10A2B800022B30DDCDF81090049B63B9314605229E
:10A2C800204600F038FB01460646504600F0F1FCF7
:10A2D80000283FF75CAD1F9B069D6FEA030B002328
:10A2E80007933146204600F00FFB002F3FF44BAE9A
:10A2F800079B2BB1BB4203D01946204600F004FB54
:10A308003946204600F000FB3DE600263746E2E7E6
:10A31800BB4637463BE5099BCDF81090002B7FF4F0
:10A3280012AF069D31465046FFF754FA069B00F1DE
:10A33800300905F8019B049AEB1A9A4200F38180D0
:10A34800069B012AACBF9B1801339846002307934C
:10A3580051460122204600F05BFC3146824600F05F
:10A36800A8FC002834DC02D119F0010F30D1454691
:10A3780015F8013C6A1E302BB3D11546F8E738466C
:10A38800FFE6012322E7029A002A04DB28D11E9A5D
:10A3980032BB089A22BB002B7FF732AF514601220D
:10A3A800204600F035FC3146824600F082FC002849
:10A3B80005DC7FF425AF19F0010F3FF421AFB9F1A7
:10A3C800390F7FF41BAF392308F1010808F8013C65
:10A3D800454615F8013C6A1E392B3AD001333FE057
:10A3E800002B08F1010505DDB9F1390FEBD009F1B2
:10A3F800010907E7069B049AEB1A9342A84605F859
:10A40800019CA5D0514600230A22204600F093FA69
:10A41800079B8246BB424FF00A024FF000030799A0
:10A42800204604D100F087FA07900746B1E600F00D
:10A4380082FA002307900A223946204600F07BFA68
:10A44800F3E7514600230A22204600F074FA8246B8
:10A4580068E7069B934205D13123069A0BF1010B5D
:10A4680013703EE71546B4E7094BFFF7A3BA229BE2
:10A47800002B7FF47DAA074BFFF79CBA049B002BA7
:10A488003FF74FAF1E9B022B7FF74BAF14E700BF80
:10A49800B8B90008DCB900088A892DE9F0410546F9
:10A4A80010070C465AD44B68002B05DC0B6C002BAC
:10A4B80002DC0020BDE8F081E66A002EF9D0002316
:10A4C80012F480522F682B6033D0606DA3895A072D
:10A4D80005D56368C01A636B0BB1236CC01A0023DF
:10A4E8000246E66A216A2846B047431CA38906D17A
:10A4F80029681D294BD82B4ACA40D60747D50022C0
:10A5080062602269D904226004D5421C01D12B68FB
:10A5180003B96065616B2F600029CAD004F1440358
:10A52800994202D0284600F09BFC00206063BDE8F9
:10A53800F081216A01232846B047411CC6D12B6807
:10A54800002BC3D01D2B01D0162B01D12F60B0E7F3
:10A55800A38943F04003A381BDE8F0810F69002F70
:10A56800A7D0930718BF00230E6808BF4B69A6EB56
:10A5780007080F608B60B8F1000F9ADD43463A4632
:10A58800216A2846A66AB047002807DCA38943F059
:10A598004003A3814FF0FF30BDE8F0810744A8EBEA
:10A5A8000008E8E70100402038B50B6905460C466D
:10A5B800DBB118B183690BB900F060F80C4B9C4211
:10A5C80009D16C68B4F90C307BB121462846BDE846
:10A5D8003840FFF761BF074B9C4201D1AC68F1E7F7
:10A5E800054B9C4208BFEC68ECE7002038BD00BF73
:10A5F8000CBA00082CBA0008ECB90008014900F0B0
:10A60800A9B800BFB1A50008002310B5044603602F
:10A618004360836081814366C281036143618361D2
:10A62800194608225C30FEF74EFA054B2462636235
:10A63800044BA362044BE362044B236310BD00BFC9
:10A64800F9B400081BB5000853B5000877B5000831
:10A6580070B568254A1E55430E4605F1740100F091
:10A668004BFC044640B1002180E842000C30A06059
:10A6780005F16802FEF727FA204670BD836910B518
:10A68800044633BB8364C3640365124B124A1B68D8
:10A698008262984204BF0123836100F01FF8606062
:10A6A800204600F01BF8A060204600F017F80022B2
:10A6B800E06004216068FFF7A7FF01220921A06874
:10A6C800FFF7A2FF02221221E068FFF79DFF012396
:10A6D800A36110BDA4B9000805A60008F8B51C4B75
:10A6E80007461E68B36913B93046FFF7C7FF4836F7
:10A6F800B4687368013B03D5336833B13668F7E74C
:10A70800B4F90C506DB16834F4E704213846FFF70A
:10A718009FFF30600028F1D10C2304463B6020469F
:10A72800F8BD4FF6FF73E38101236566A3812560B9
:10A73800A560656025616561A5610822294604F167
:10A748005C00FEF7C0F96563A563A564E564E6E708
:10A75800A4B900082DE9F84380468946002600F18F
:10A76800480414B93046BDE8F883A5686768013F16
:10A7780001D52468F5E7AB89012B07D9B5F90E3067
:10A78800013303D029464046C84706436835EEE7FB
:10A79800044B1B68186A044B002808BF1846F030A1
:10A7A800704700BF0C0000207000002070B50E46F6
:10A7B800B1F90E1090B0002914461D4607DA00239F
:10A7C8002B60B3891A0610D44FF480630EE001AAF7
:10A7D80000F0F4FE0028F2DB029A02F47042A2F5BF
:10A7E80000535A425A412A60EEE740230020236072
:10A7F80010B070BD8B8973B59D0706460C4607D50A
:10A8080004F14703236023610123636102B070BD33
:10A8180001AB6A46FFF7CAFF00990546304600F0CB
:10A828006BFB48B9B4F90C309A05EFD423F0030355
:10A8380043F00203A381E3E70D4BB362A3892060D1
:10A8480043F08003A381009B20616361019B5BB19E
:10A85800B4F90E10304600F0C3FE28B1A38923F0E6
:10A86800030343F00103A381A3891D43A581CDE719
:10A8780005A60008024B0146186800F03DBB00BF62
:10A888000C00002010B5C9B202449042034601D121
:10A89800002010BD1C7801308C42F6D1184610BD3E
:10A8A80070B5456A04460E463DB91020FFF7E2FF31
:10A8B8006062456085600560C560656AEB6883B164
:10A8C800636ADB6853F82600B8B9012101FA06F576
:10A8D8006A1D9200204600F0B4FA60B146608560B7
:10A8E8000EE021220421204600F0ABFA636AE860FA
:10A8F800DB68002BE4D1002070BD026843F82620F5
:10A9080000230361C36070BD70B5446A06460D46F6
:10A918003CB91020FFF7AEFF7062446084600460A9
:10A92800C4603DB1736A6A68DB6853F82210296015
:10A9380043F8225070BD2DE9F0411F4606460C46EB
:10A9480000230D6901F1140EDEF80000013381B215
:10A9580002FB0171000C0F0C02FB007089B201EBC5
:10A9680000419D424FEA10474EF8041BECDCD7B17A
:10A97800A3689D4212DB616830460131FFF790FF02
:10A988008046226904F10C01023292000C30FEF775
:10A998008FF821463046FFF7B7FF444604EB85039E
:10A9A80001355F6125612046BDE8F081020C120483
:10A9B8000346B2B90304102013F07F4F04BF1B02F3
:10A9C800083013F0704F04BF1B01043013F0404FE0
:10A9D80004BF9B000230002B06DB5B0003D501306F
:10A9E80070470020E8E7202070470368014613F00D
:10A9F80007020BD0DA0723D4980749BF5B089B08E6
:10AA080001200B605CBF0B600220704798B2A8B9A8
:10AA180010201B0C13F0FF0F04BF1B0A08301A0785
:10AA280004BF1B0904309A0704BF9B080230DA07E9
:10AA380002D45B0806D001300B6070471046E9E786
:10AA4800002070472020704710B50C460121FFF701
:10AA580027FF01224461026110BD2DE9F74F14461A
:10AA68000A69236989469A42BEBF0B46A1461C461D
:10AA7800D9F81070D4F810A0D9F80830D9F8041013
:10AA880007EB0A069E42C8BF0131FFF709FF00F134
:10AA980014052B46002205EB8608434516D304F11E
:10AAA800140209F1140102EB8A0301EB87070193F1
:10AAB800019C134694420CD8002E03DD58F8043D3F
:10AAC800002B54D0066103B0BDE8F08F43F8042B87
:10AAD800E3E7B3F800A00432BAF1000F20D0AE4685
:10AAE80089464FF0000C59F8044BBEF800B0A3B2E9
:10AAF8000AFB03B34FEA144BDEF8004063444FEA05
:10AB0800144C0AFB0BC404EB13449BB243EA044302
:10AB18004F454FEA144C4EF8043BE4D8CEF800C039
:10AB280032F8029CB9F1000F1FD0AE468C464FF0A8
:10AB3800000A2B68BCF80040BEF802B09BB209FBC3
:10AB480004B4A24443EA0A434EF8043B5CF8043BCD
:10AB5800BEF800401B0C09FB0343674503EB1A438F
:10AB68004FEA134AE6D8CEF800300435A0E7013E94
:10AB7800A2E700002DE9F843154612F00302064645
:10AB88000F4607D0214C013A002354F82220FFF742
:10AB9800D2FE0746AD1035D0746A3CB91020FFF7D5
:10ABA80069FE7062446084600460C460D6F82480E2
:10ABB800D8F808404CB940F271213046FFF744FFFD
:10ABC80000230446C8F8080003604FF00008EB07AC
:10ABD8000AD5394622463046FFF73FFF81463946B7
:10ABE8003046FFF791FE4F466D100BD0206838B9FC
:10ABF800224621463046FFF730FF2060C0F800802B
:10AC08000446E4E73846BDE8F88300BF40BB0008C7
:10AC18002DE9F0470C460746164623694FEA621AA3
:10AC28000AEB03094968A36809F10105AB4231DB66
:10AC38003846FFF735FE00228046114600F114031E
:10AC480052452ADB20692AEAEA7A04F1140116F04F
:10AC58001F0203EB8A0301EB800E22D00020C2F111
:10AC6800200C0E689640304343F8040B51F8040B4F
:10AC78008E4520FA0CF0F4D8186008B109F10205E5
:10AC8800013D3846C8F810502146FFF73DFE4046C2
:10AC9800BDE8F08701315B00C8E743F822100132B4
:10ACA800CEE7043B51F8042B8E4543F8042FF9D81E
:10ACB800E6E703690A6930B59B1A0CD19200143093
:10ACC80014318418114454F8045D51F8042D954248
:10ACD80003D005D30123184630BDA042F3D3FAE7C9
:10ACE8004FF0FF33F7E72DE9F0470D4607461146C9
:10ACF80028461446FFF7DDFF061E08D131463846C0
:10AD0800FFF7CEFD012346610361BDE8F087A4BFCC
:10AD180023462C4638466168A6BF1D4600260126F4
:10AD2800FFF7BEFD4FF0000CC6602B69266904F1E1
:10AD3800140205F1140902EB860709EB830800F1F8
:10AD4800140152F804AB59F8045B1FFA8AF3634400
:10AD5800ACB21B1B2C0CC4EB1A4404EB23449BB26F
:10AD68004FEA244CC84543EA0444964641F8044B4C
:10AD7800E7D8BE4505D351F8043D8BB10661BDE85F
:10AD8800F0875EF8044BA2B26244131403EB144339
:10AD980092B242EA03424FEA234C41F8042BE8E717
:10ADA800013EE8E72DE9F3411C4601219046089E43
:10ADB800099DFFF775FDC4F31302C4F30A5407464F
:10ADC80034BB0192B8F1000F27D002A840F8088DD3
:10ADD800FFF70BFE0099F0B1019AC0F1200302FAC7
:10ADE80003F30B43C2407B610192019B002B14BF0C
:10ADF80002210121BB613961C4B1A4F23344044486
:10AE08003460C0F135002860384602B0BDE8F081F2
:10AE180042F48012D5E77961E7E701A8FFF7E5FD7D
:10AE28000121019B39617B612030E5E7A0F23240C6
:10AE380007EB810330601869FFF7B8FDC0EB4110DC
:10AE4800E1E738B502FB01F4214600F055F8054664
:10AE580018B122460021FDF736FE284638BD00000D
:10AE680038B50546002943D051F8043C0C1F002B87
:10AE7800B8BFE41800F002FC1E4A1368104633B944
:10AE8800636014602846BDE8384000F0F8BBA34270
:10AE98000BD921686218934201BF1A685B6852187F
:10AEA800226063600460EDE713465A680AB1A24263
:10AEB800FAD919685818A0420BD1206801445818CB
:10AEC80082421960DED110685268014419605A60E4
:10AED800D8E702D90C232B60D4E7206821188A42CE
:10AEE80001BF116852680918216062605C60C9E797
:10AEF80038BD00BF8802002070B5CD1C25F00305C1
:10AF080008350C2D38BF0C25002D064601DBA9425B
:10AF180003D90C233360002070BD00F0AFFB234A37
:10AF28001468214691B9224C23681BB9304600F0B9
:10AF3800CFFA20602946304600F0CAFA431C26D1D1
:10AF48000C233046336000F09AFBE4E70B685B1B88
:10AF58001AD40B2B0FD90B60CC18CD50304600F00B
:10AF68008EFB04F10B00231D20F00700C31A1BD031
:10AF78005A42E25070BD8C420BBF63684B68136045
:10AF8800636018BF0C46E9E70C464968CAE7C41C69
:10AF980024F00304A04205D0211A304600F098FAA4
:10AFA8000130CDD02560D9E770BD00BF88020020F0
:10AFB8008C0200202DE9F0478E6882469E420C469E
:10AFC8009146984635D88A8912F4906F31D0022379
:10AFD800256809696F1A656905EB450595FBF3F561
:10AFE80008F101033B449D4238BF1D46530531D546
:10AFF8002946FFF781FF064650B90C23CAF80030EE
:10B00800A3894FF0FF3043F04003A381BDE8F087E8
:10B018003A462169FDF74CFDA38923F4906343F078
:10B028008003A38126613E44266046466561ED1B88
:10B03800A560464528BF464649463246206800F086
:10B0480003FBA36800209B1BA36023681E442660A3
:10B05800BDE8F0872A4600F013FB06460028E1D138
:10B0680021695046FFF7FCFEC7E700002DE9F04FC5
:10B078009DB003938B8980461C060D4616460FD556
:10B088000B696BB94021FFF737FF2860286128B9A1
:10B098000C23C8F800304FF0FF30C4E040236B6148
:10B0A8000023099320238DF8293030234FF0010B1A
:10B0B8008DF82A3037463C4614F8013B002B3CD12A
:10B0C800B7EB060A0BD05346324629464046FFF7EF
:10B0D80071FF013000F0A280099B534409933B782B
:10B0E800002B00F09B8000234FF0FF32049307935E
:10B0F800059206938DF853301A930522217850480B
:10B10800FFF7C0FB671C049BD8B9D90644BF2022AF
:10B118008DF853201A0744BF2B228DF8532022782C
:10B128002A2A16D000210A20079A27463B7801349C
:10B13800303B092B50D9C9B111E0252BC0D0274687
:10B14800B9E73F4A3C46801A0BFA00F018430490CE
:10B15800D3E7039A111D12680391002A01DB0792B5
:10B1680004E0524243F00203079204933B782E2BEB
:10B178000DD17B78791C2A2B32D1039B02371A1DFB
:10B188001B680392002BB8BF4FF0FF3305932D4C7B
:10B19800032239782046FFF775FB38B14023001B9E
:10B1A80003FA00F0049B013703430493397806221D
:10B1B80025487E1C8DF82810FFF764FB002835D041
:10B1C800224BFBB9039B073323F007030833039390
:10B1D800099B4B4409936DE700FB02320121A4E768
:10B1E80000230A24184605930F463A780131303A6D
:10B1F800092A03D9002BCAD00590C8E704FB002010
:10B208000123F1E703AB00932A46114B04A94046FA
:10B21800FDF7F2FCB0F1FF3F8146D9D1AB895B065F
:10B228003FF539AF09981DB0BDE8F08F03AB009327
:10B238002A46074B04A94046FDF78EFFEAE700BF00
:10B248004CBB000852BB000856BB0008018C000824
:10B25800BDAF0008936810B4013B002B936008DA77
:10B268009469A34202DBCBB20A2B02D110BCFEF7D1
:10B27800F1B91368581C10601970C8B210BC704737
:10B28800F8B506460F461446D518AC4201D1002041
:10B2980007E03A4614F8011B3046FFF7DBFF431C72
:10B2A800F3D1F8BD2DE9F04F9DB00C461746039336
:10B2B800064618B183690BB9FFF7E0F97C4B9C424D
:10B2C80057D17468A38918075DD52369002B5AD014
:10B2D8000023099320238DF8293030234FF0010BE8
:10B2E8008DF82A30B846454615F8013B002B55D154
:10B2F800B8EB070A0BD053463A4621463046FFF7CB
:10B30800BFFF013000F0C480099B5344099398F8AB
:10B318000030002B00F0BC8000234FF0FF32049374
:10B328000793059206938DF853301A9305222978CE
:10B338006048FFF7A7FA05F10108049B002831D1FE
:10B34800D90644BF20228DF853201A0744BF2B2268
:10B358008DF853202A782A2A2CD000210A20079A0F
:10B36800A84698F800300135303B092B6DD971B3E8
:10B3780026E0514B9C4201D1B468A3E74F4B9C4255
:10B3880008BFF4689EE721463046FEF7B5F9002865
:10B398009ED04FF0FF301DB0BDE8F08F252BA7D011
:10B3A800A846A0E7434A4546801A0BFA00F018431E
:10B3B8000490BBE7039A111D12680391002A01DB70
:10B3C800079204E0524243F002030792049398F86C
:10B3D80000302E2B10D198F8013008F101012A2BEA
:10B3E80037D1039B08F102081A1D1B680392002B32
:10B3F800B8BF4FF0FF330593314D032298F8001082
:10B408002846FFF73FFA40B14023401B03FA00F0FB
:10B41800049B08F101080343049398F800100622DE
:10B42800284808F101078DF82810FFF72BFA0028A3
:10B4380034D0254B03BB039B073323F007030833A2
:10B448000393099B4B4409934CE700FB023201210B
:10B4580086E700230A2518460593884698F80020B1
:10B468000131303A092A03D9002BC5D00590C3E72A
:10B4780005FB00200123F0E703AB00932246134BA2
:10B4880004A93046FDF7B8FBB0F1FF3F8146D8D19B
:10B49800A3895B063FF57DAF09987CE703AB009372
:10B4A80022460A4B04A93046FDF756FEECE700BFDA
:10B4B8000CBA00084CBB00082CBA0008ECB900080C
:10B4C80052BB000856BB0008018C000889B200086E
:10B4D80038B50023054C054608462360FDF708FAF1
:10B4E800431C02D1236803B12B6038BD50180020DB
:10B4F80010B50C46B1F90E1000F0E8F80028ABBF03
:10B50800636DA3891B1823F48053ACBF6365A381C3
:10B5180010BD2DE9F0411F468B890546DB050C4619
:10B52800164605D502230022B1F90E1000F068F87E
:10B53800A389324623F48053A381B4F90E103B4605
:10B548002846BDE8F04100F017B810B50C46B1F92F
:10B558000E1000F055F8431CA38915BF606523F44D
:10B56800805343F48053A38118BFA38110BDB1F960
:10B578000E1000F013B8000038B50546084611460D
:10B588000022054C22601A46FCF70EFC431C02D12F
:10B59800236803B12B6038BD5018002038B500234C
:10B5A800054C054608462360FDF7BCF9431C02D14B
:10B5B800236803B12B6038BD5018002038B500232C
:10B5C800064C0546084611462360FDF7AEF9431CB4
:10B5D80002D1236803B12B6038BD00BF501800208A
:10B5E80038B50023054C054608462360FDF7A2F947
:10B5F800431C02D1236803B12B6038BD50180020CA
:10B6080038B50546084611460022054C22601A4600
:10B61800FDF792F9431C02D1236803B12B6038BDB2
:10B628005018002082B001B901A942B14BB113787A
:10B638000B601278101C18BF012002B0704710462A
:10B64800FBE76FF00100F8E7884210B501EB020351
:10B6580003D8421E99420CD110BD9842F9D28118E4
:10B66800D21AD34200D110BD13F8014D01F8014D93
:10B67800F7E711F8014B02F8014FEBE77047704705
:10B68800F8B5074614460E4621B91146BDE8F840FC
:10B69800FFF732BC22B9FFF7E3FB25462846F8BD81
:10B6A80000F033F884420FD921463846FFF724FCCE
:10B6B80005460028F2D031462246FDF7F9F9314611
:10B6C8003846FFF7CDFBE9E73546E7E738B50546E5
:10B6D800084611460022054C22601A46FDF7FAF882
:10B6E800431C02D1236803B12B6038BD50180020D9
:10B6F80049B1FF2A8BBF8A230A700360012088BFE3
:10B708004FF0FF3070470846704751F8040C002886
:10B71800A0F10400BCBF0B58C0187047F8B500BFB3
:10B72800F8BC08BC9E467047F8B500BFF8BC08BC1A
:04B738009E46704772
:10B7400000061016000610164368616E6E656C20C8
:10B7500053657474696E6700707265737320616EEF
:10B760007920427574746F6E0064617461203A20B0
:10B7700025662020206F6666736574203A20202598
:10B78000660D0A00202032387E32382E3520474898
:10B790007A202000202032382E357E32392047484A
:10B7A0007A2000202032397E32392E352047487ADF
:10B7B0002000202032392E357E33302047487A2031
:10B7C0000020202020322E3447487A2020202020BC
:10B7D0000020202020352E3847487A2020202020A5
:10B7E00000202041204368203135304D487A200028
:10B7F000202020202530362E326620202064420072
:10B800002020204120436820333047002020204161
:10B81000204368616E6E656C20202000202020206F
:10B8200053657474696E67002020204120436820AE
:10B8300057494649202000202042204368203135C6
:10B84000304D487A200020202042204368203330A9
:10B850004700202042204368616E6E656C00202006
:10B8600042204368205749464920200043726974AA
:10B870006963616C204572726F720D005B45727274
:10B880006F72205D446566616C757420696E202559
:10B89000732020202020204C494E45203A2564204A
:10B8A0000D0A00417474656E5F4F70657261746556
:10B8B0005F4D656D5F525700427574746F6E5F50D7
:10B8C0005245535320455343200D0A00427574746A
:10B8D0006F6E5F5052455353204D454E55200D0A13
:10B8E00000427574746F6E5F554E5052455353202D
:10B8F0004D454E55200D0A00427574746F6E5F55AC
:10B9000050205052455353200D0A00427574746FF5
:10B910006E5F555020554E5052455353200D0A002E
:10B9200048414C5F4750494F5F455854495F436118
:10B930006C6C6261636B00253032782000434845AF
:10B94000434B53554D5F4552524F52202052656331
:10B9500076435243203A202530327820202C20692B
:10B960006E6465782025640D0A005768617420486C
:10B97000617070656E3F0D004C4F4E47204B45592E
:10B980002050524553530D6D000000000000000090
:10B990000001020304060708090000000001020379
:10B9A0000400000010000020494E4600696E660049
:10B9B0004E414E006E616E0030003031323334350E
:10B9C000363738394142434445460030313233340A
:10B9D000353637383961626364656600496E666979
:10B9E0006E697479004E614E000000000000000096
:10B9F0000000000000000000000000000000000047
:10BA00000000000000000000000000000000000036
:10BA10000000000000000000000000000000000026
:10BA20000000000000000000000000000000000016
:10BA30000000000000000000000000000000000006
:10BA400000000000000000000000000000000000F6
:10BA50000080E03779C34143176E05B5B5B893460A
:10BA6000F5F93FE9034F384D321D30F94877825AD6
:10BA70003CBF737FDD4F1575000000000000F03FF4
:10BA800000000000000024400000000000005940B9
:10BA90000000000000408F40000000000088C3400C
:10BAA00000000000006AF8400000000080842E4181
:10BAB00000000000D01263410000000084D79741CD
:10BAC0000000000065CDCD41000000205FA00242D3
:10BAD000000000E876483742000000A2941A6D4248
:10BAE000000040E59C30A2420000901EC4BCD6423B
:10BAF00000003426F56B0C430080E03779C34143E6
:10BB000000A0D8855734764300C84E676DC1AB435B
:10BB1000003D9160E458E143408CB5781DAF154479
:10BB200050EFE2D6E41A4B4492D54D06CFF0804454
:10BB3000F64AE1C7022DB544B49DD9794378EA4469
:10BB400005000000190000007D000000232D302BAF
:10BB50002000686C4C00656667454647004300500E
:10BB60004F534958002E0000202020202020202064
:10BB7000202828282828202020202020202020209D
:10BB800020202020202020208810101010101010BD
:10BB90001010101010101010040404040404040405
:10BBA0000404101010101010104141414141410196
:10BBB0000101010101010101010101010101010175
:10BBC0000101011010101010104242424242420284
:10BBD0000202020202020202020202020202020245
:10BBE00002020210101010200000000000000000EF
:10BBF0000000000000000000000000000000000045
:10BC00000000000000000000000000000000000034
:10BC10000000000000000000000000000000000024
:10BC20000000000000000000000000000000000014
:10BC30000000000000000000000000000000000004
:10BC400000000000000000000000000000000000F4
:10BC500000000000000000000000000000000000E4
:08BC60000000000000000000DC
:08BC68000852FF7F01000000FB
:04BC7000AD0100081A
:04BC7400890100083A
:10BC780001000000100000000024F4001000002063
:10BC8800000000000CBA00082CBA0008ECB9000843
:10BC9800000000000000000000000000000000009C
:10BCA800000000000000000000000000000000008C
:10BCB800000000000000000000000000000000007C
:10BCC800000000000000000000000000000000006C
:10BCD800000000000000000000000000000000005C
:10BCE8004300000000000000000000000000000009
:10BCF800000000000000000000000000000000003C
:10BD080043000000000000000000000000000000E8
:10BD1800000000000000000000000000000000001B
:10BD280043000000000000000000000000000000C8
:10BD380000000000000000000000000000000000FB
:10BD480043000000000000000000000000000000A8
:10BD580000000000000000000000000000000000DB
:10BD68004300000000000000000000000000000088
:10BD780000000000000000000000000000000000BB
:10BD88004300000000000000000000000000000068
:10BD9800000000000000000000000000000000009B
:10BDA8004300000000000000000000000000000048
:10BDB800000000000000000000000000000000007B
:10BDC800F9B600082DB600080000000067BB00089F
:10BDD80065BB0008CBB80008CBB80008CBB8000892
:10BDE800CBB80008CBB80008CBB80008CBB800081F
:10BDF800CBB80008CBB80008FFFFFFFFFFFFFFFF2D
:10BE0800FFFFFFFFFFFF00000100415343494900C6
:10BE1800000000000000000000000000000000001A
:10BE280000000000000000000000415343494900A1
:10BE380000000000000000000000000000000000FA
:0CBE4800000000000000000000000000EE
:0400000508008A1154
:00000001FF
